:020000040000FA
:0600000057EF4CF0120066
:0A000600040054990000C10400003A
:100010003A000000F7980000210F000001000000E6
:1000200017990000840400003D000000FC980000C7
:08003000E10000001B000000CC
:08003800D9CFE6FFDACFE6FFA5
:10004000E1CFD9FFE2CFDAFFE652E652FC0EDBCF7A
:10005000DEFFDBCFDDFFF80EDBCF00F0DB06F90EB5
:10006000DBCF01F001E2DB06005001100CE0DFCF36
:10007000E9FFDF2A010EDBCFEAFF01E3DB2AFA0EFC
:10008000DBCFEFFFE8D7E552E552E552E5CFDAFFE7
:10009000E7CFD9FF1200D9CFE6FFDACFE6FFE1CFF5
:1000A000D9FFE2CFDAFF060EE12402E3E168E6526F
:1000B000E16EFC0EDBCFDEFFDBCFDDFFFA0EDBCF28
:1000C0003FF0FB0EDBCF40F0020E3FC0DBFF030E24
:1000D00040C0DBFF040EDB6A050EDB6AF80EDBCFE7
:1000E00000F0DB06F90EDBCF01F001E2DB06005089
:1000F000011022E0DFCFE9FFDF2A010EDBCFEAFFAC
:1001000001E3DB2AEFCF04F0020EDBCFE9FFDB2AAD
:10011000030EDBCFEAFF01E3DB2AEF50045C026E43
:10012000036A02BE0368040E02C0DBFF050E03C0B3
:10013000DBFF02500310D2E0040EDBCF00F0050E0F
:10014000DBCF01F000C0F3FF01C0F4FF060EE15C5D
:1001500002E2E16AE552E16EE552E5CFDAFFE7CF70
:10016000D9FF1200D9CFE6FFDACFE6FFE1CFD9FF02
:10017000E2CFDAFF0C0EE12402E3E168E652E16E21
:100180000A0EFEC4DBFF0B0EFFC4DBFFD950FA0FD3
:10019000E96EFF0EDA20EA6E020EEE5C000EEE58FB
:1001A000000EEE58000EEE5801E27FD2FA0EDBCFC1
:1001B00000F0FB0EDBCF01F0FC0EDBCF02F0FD0EFA
:1001C000DBCF03F00A0EDBCFE9FF0B0EDBCFEAFF3C
:1001D000060EE926000EEA22EE50005CEE500158B1
:1001E000EE500258EE50035801E35FD20A0EDBCF07
:1001F000E9FF0B0EDBCFEAFFEF50030A01E1ACD1C0
:10020000010A01E146D1030A01E04FD2FA0EDBCF29
:100210003FF0FB0EDBCF40F0020E3FC0DBFF030ED2
:1002200040C0DBFF020EDBCF00F0030EDBCF01F09E
:10023000010E0F0B05E0D89001320032E806FBE119
:10024000D950020FE96E000EDA20EA6E0050EE2659
:100250000150ED22020EDBCF00F0030EDBCF01F0E8
:100260000001010E0116040E00C0DBFF050E01C0E7
:10027000DBFFD950020FE96E000EDA20EA6E090E9C
:100280000F0B06E0EC52D890ED32EF32E806FAE1BF
:10029000D950040FE96E000EDA20EA6EFF0EEE1858
:1002A00002E1010EED183FE0020EE66EE66A040E72
:1002B000DBCFE6FF050EDBCFE6FF020EDBCF00F063
:1002C000030EDBCF01F0026A036A0A0EDBCFE9FFFF
:1002D0000B0EDBCFEAFF0A0EE926000EEA22EE50F3
:1002E0000026EE500122EE500222EE50032200C002
:1002F000E6FF01C0E6FF02C0E6FF03C0E6FFD950FB
:10030000060FE66E000EDA20E66E0AEC42F0046E8E
:100310000A0EE15C02E2E16AE552E16E0450000976
:1003200001E17FD0C2D1010EE66EE66AE668E66EB4
:10033000020EDBCF00F0030EDBCF01F0026A036A8E
:100340000A0EDBCFE9FF0B0EDBCFEAFF0A0EE92630
:10035000000EEA22EE500026EE500122EE5002225C
:10036000EE50032200C0E6FF01C0E6FF02C0E6FF38
:1003700003C0E6FFD950060FE66E000EDA20E66EE7
:100380000AEC42F0046E0A0EE15C02E2E16AE55218
:10039000E16E0450000901E088D1010EE66EE66AC4
:1003A000000EE66EE66A020EDBCF04F0030EDBCF32
:1003B00005F0066A076A0A0EDBCFE9FF0B0EDBCFFA
:1003C000EAFF0A0EE926000EEA22EE500424006E2F
:1003D000EE500520016EEE500620026EEE50072012
:1003E000036E002A000E01220222032200C0E6FF53
:1003F00001C0E6FF02C0E6FF03C0E6FFD950070FC9
:10040000E66E000EDA20E66E0AEC42F0086E0A0E86
:10041000E15C02E2E16AE552E16E0850000901E0A8
:1004200044D1070EDBCF02F002C003F0026A060ED1
:10043000DB500210DE6E03C0DDFF010E046E056AA4
:10044000066A076AD950FA0FE96EFF0EDA20EA6EE3
:10045000EE500416EE500516EE500616EE50071636
:1004600004500510061007100BE0DECF00F0DDCFC2
:1004700001F0040ED89001320032E804FBE169D0AB
:10048000DECF00F0DDCF01F0FF0E00160F0E0116DB
:1004900060D0020EE66EE66AFA0EDBCF00F0FB0ECD
:1004A0000001016A010ED89000360136E806FBE132
:1004B00000C0E6FF01C0E6FFFA0EDBCF02F0FB0E44
:1004C000DBCF03F0FC0EDBCF04F0FD0EDBCF05F03D
:1004D000080ED8900532043203320232E806F9E100
:1004E0000A0EDBCFE9FF0B0EDBCFEAFF0A0EE9268F
:1004F000000EEA22EE500226EE500322EE500422B5
:10050000EE50052202C0E6FF03C0E6FF04C0E6FF8E
:1005100005C0E6FFD950060FE66E000EDA20E66E43
:100520000AEC42F0066E0A0EE15C02E2E16AE55274
:10053000E16E0650000901E0B8D0070EDBCF04F0F1
:1005400004C005F0046A060EDB500410006E05C0FE
:1005500001F0026A036AA0D0040EE66EE66AFA0EA3
:10056000DBCF00F0FB0E0001016A009E020ED89066
:1005700000360136E806FBE100C0E6FF01C0E6FFF9
:10058000FA0EDBCF02F0FB0EDBCF03F0FC0EDBCF6D
:1005900004F0FD0EDBCF05F0070ED89005320432D3
:1005A00003320232E806F9E10A0EDBCFE9FF0B0E57
:1005B000DBCFEAFF0A0EE926000EEA22EE50022601
:1005C000EE500322EE500422EE50052202C0E6FF58
:1005D00003C0E6FF04C0E6FF05C0E6FFD950060FE2
:1005E000E66E000EDA20E66E0AEC42F0066E0A0EA7
:1005F000E15C02E2E16AE552E16E0650000955E174
:10060000090EDBCF04F0056A066A076A180E1F0B95
:1006100007E0D8900436053606360736E806F9E1D5
:10062000080EDBCF08F0096A0A6A0B6A100E1F0B6E
:1006300007E0D890083609360A360B36E806F9E1A5
:1006400008500412095005120A5006120B500712E6
:10065000070EDBCF0CF00CC00DF00C6A0E6A0F6AAF
:100660000C5004120D5005120E5006120F500712B6
:10067000060EDBCF10F0116A126A136A04501010D4
:10068000006E05501110016E06501210026E0750D8
:100690001310036E0F0E031600C03DF001C03EF0B4
:1006A00002C03FF003C040F005D0010E3D6E3E6A2F
:1006B0003F6A406A0C0EE15C02E2E16AE552E16EDB
:1006C000E552E5CFDAFFE7CFD9FF1200D9CFE6FF39
:1006D000DACFE6FFE1CFD9FFE2CFDAFFE652E6520A
:1006E000FEC4DEFFFFC4DDFFD950FA0FE96EFF0E36
:1006F000DA20EA6E020EEE5E000EEE5AEE5AEE5A66
:10070000DECFE9FFDDCFEAFF060EE926000EEA2282
:10071000EECF00F0EECF01F0EECF02F0EFCF03F01E
:10072000020E005E000E015A025A035AD950FA0F07
:10073000E96EFF0EDA20EA6E0050EE5C0150EE58D2
:100740000250EE580350EE5805E33D6A3E6A3F6A98
:10075000406A46D0DECFE9FFDDCFEAFF120EE92680
:10076000000EEA22EECF08F0EECF09F0EECF0AF04D
:10077000EFCF0BF0DECFE9FFDDCFEAFF020EE92677
:10078000000EEA22EFCF04F0056A066A076A04C089
:100790003DF005C03EF006C03FF007C040F0FA0E45
:1007A000DBCF42F0FB0EDBCF43F0FC0EDBCF44F09F
:1007B000FD0EDBCF45F085EC4BF039500824006E80
:1007C0003A500920016E3B500A20026E3C500B202B
:1007D000036E00C03DF001C03EF002C03FF0406E2D
:1007E000E552E552E552E5CFDAFFE7CFD9FF120037
:1007F000D9CFE6FFDACFE6FFE1CFD9FFE2CFDAFFCC
:10080000060EE12402E3E168E652E16E040EFEC446
:10081000DBFF050EFFC4DBFFFC0EDBCFE9FFFD0EA7
:10082000DBCFEAFFEE6AED6AFC0EDBCFE9FFFD0EDF
:10083000DBCFEAFF040EE926000EEA22EECFDFFF4F
:10084000010EEECFDBFF020EEECFDBFF030EEECF8D
:10085000DBFFD9CFE9FFDACFEAFF010EEE1805E1A1
:10086000EE5003E1EE5001E1EE501FE0040EDBCF4D
:10087000E9FF050EDBCFEAFF060EE926000EEA22AD
:10088000EECF00F0EECF01F0EECF02F0EFCF03F0AD
:10089000D9CFE9FFDACFEAFF0050EE5C0150EE5805
:1008A0000250EE580350EE5802E3010E93D0D9CF18
:1008B000E9FFDACFEAFFEECF00F0EECF01F0EECFA6
:1008C00002F0EFCF03F000500110021003101EE100
:1008D000040EDBCFE9FF050EDBCFEAFFEF50030884
:1008E00015E1040EDBCFE9FF050EDBCFEAFF0E0EAC
:1008F000E926000EEA22EECFDFFF010EEECFDBFF8E
:10090000020EEECFDBFF030EEECFDBFFFC0EDBCFE4
:10091000E9FFFD0EDBCFEAFF080EE926000EEA2212
:10092000DFCFEEFF010EDBCFEEFF020EDBCFEEFFDF
:10093000030EDBCFEEFFD9CFE9FFDACFEAFFEECF30
:1009400004F0EECF05F0EECF06F0EFCF07F0045045
:100950000510061007101AE0D9CFE9FFDACFEAFF39
:10096000EECFE6FFEECFE6FFEECFE6FFEFCFE6FFFE
:10097000ADDEE552E552E552E5523DC000F03EC025
:1009800001F03FC002F040C003F012D0040EDBCFF4
:10099000E9FF050EDBCFEAFF0E0EE926000EEA2284
:1009A000EECF00F0EECF01F0EECF02F0EFCF03F08C
:1009B000FC0EDBCFE9FFFD0EDBCFEAFF0C0EE926D4
:1009C000000EEA2200C0EEFF01C0EEFF02C0EEFF03
:1009D00003C0EEFF006E060EE15C02E2E16AE55242
:1009E000E16E0050E552E5CFDAFFE7CFD9FF120004
:1009F000D9CFE6FFDACFE6FFE1CFD9FFE2CFDAFFCA
:100A0000080EE12402E3E168E652E16E060EFEC440
:100A1000DBFF070EFFC4DBFFFC0EDBCFE9FFFD0EA3
:100A2000DBCFEAFFEECF00F0EFCF01F0010E0026A2
:100A3000000E0122040E00C0DBFF050E01C0DBFF2B
:100A4000D950040FE96E000EDA20EA6EEE50ED1078
:100A500001E1D5D0FC0EDBCFE9FFFD0EDBCFEAFFD5
:100A60000C0EE926000EEA22EECF00F0EECF01F0E8
:100A7000EECF02F0EFCF03F0005001100210031090
:100A800001E1BDD0040EDBCF00F0050E016A0F0EB0
:100A900000160050011001E0F2D0FC0EDBCFE9FFA0
:100AA000FD0EDBCFEAFF0C0EE926000EEA22EE2A4D
:100AB000EE22EE22EE22FC0EDBCFE9FFFD0EDBCFB5
:100AC000EAFF080EE926000EEA22EECF00F0EECF94
:100AD00001F0EECF02F0EFCF03F000500110021052
:100AE00003101BE1040EDBCF00F0050EDBCF01F09D
:100AF000060EDBCFE9FF070EDBCFEAFF040EE92687
:100B0000000EEA22EECF02F0EFCF03F00250005CBD
:100B10000350015801E2B3D072D0040EDBCF02F0D3
:100B2000050EDBCF03F0040E0F0B05E0D890033267
:100B30000232E806FBE1060EDBCFE9FF070EDBCF52
:100B4000EAFF020EE926000EEA22EF040001021479
:100B5000006E016AE850011001E091D0FC0EDBCF7D
:100B6000E9FFFD0EDBCFEAFF080EE926000EEA22C0
:100B7000EECFE6FFEECFE6FFEECFE6FFEFCFE6FFEC
:100B8000B2EC00F0E552E552E552E5523DC0DEFF21
:100B90003EC0DEFF3FC0DEFF40C0DDFFDD52DD5264
:100BA000D9CFE9FFDACFEAFFD880010EEE54000E6C
:100BB000EE54000EEE54000EEE5402E3010E6CD023
:100BC000060EDBCFE9FF070EDBCFEAFF060EE926B4
:100BD000000EEA22EECF00F0EECF01F0EECF02F0F1
:100BE000EFCF03F0D9CFE9FFDACFEAFF0050EE5C98
:100BF0000150EE580250EE580350EE5802E3030E37
:100C00004BD0FC0EDBCFE9FFFD0EDBCFEAFF080E79
:100C1000E926000EEA22DFCFEEFF010EDBCFEEFF6A
:100C2000020EDBCFEEFF030EDBCFEEFFD9CFE9FFE5
:100C3000DACFEAFFEECFE6FFEECFE6FFEECFE6FF3C
:100C4000EFCFE6FF43DDE552E552E552E5523EC007
:100C500001F03FC002F040C003F0FC0EDBCFE9FF23
:100C6000FD0EDBCFEAFF0C0EE926000EEA223DC0A6
:100C7000EEFF01C0EEFF02C0EEFF03C0EEFFFC0E70
:100C8000DBCFE9FFFD0EDBCFEAFF040EDBCFEEFF8B
:100C9000050EDBCFEDFF000E006E080EE15C02E2F8
:100CA000E16AE552E16E0050E552E5CFDAFFE7CFA9
:100CB000D9FF1200D9CFE6FFDACFE6FFE1CFD9FFA7
:100CC000E2CFDAFFE652E652FC0EDBCFE6FFFD0E86
:100CD000DBCFE6FF8DDDE552E552DF6EDF5002E04F
:100CE000DF5098D0200EE66EE66AFC0EDBCFE9FFFF
:100CF000FD0EDBCFEAFFEECF00F0EFCF01F00001F9
:100D0000016A0F0E0016050ED89000360136E8066F
:100D1000FBE100C0E6FF01C0E6FFFC0EDBCFE9FF10
:100D2000FD0EDBCFEAFF0C0EE926000EEA22EECF25
:100D3000E6FFEECFE6FFEECFE6FFEFCFE6FFFA0EDF
:100D4000DBCFE6FFFB0EDBCFE6FF0AEC42F0026EE4
:100D50000A0EE15C02E2E16AE552E16E025000092E
:100D600002E0010E01D0000EDF6EDF5052E1FA0EFC
:100D7000DBCFE9FFFB0EDBCFEAFF010EEFCFDBFF9E
:100D8000DB5003E1030EDF6E44D00B0EE76EFA0E6C
:100D9000DBCFE9FFFB0EDBCFEAFFE750E926000ED1
:100DA000EA22EF50080B28E10B0EE66EE66AFC0E15
:100DB000DBCFE9FFFD0EDBCFEAFF020EE926000ED6
:100DC000EA22EECFE6FFEFCFE6FFFA0EDBCFE6FF3B
:100DD000FB0EDBCFE6FF4BEC00F0026E060EE15C93
:100DE00002E2E16AE552E16E0250F3CF00F0F4CF87
:100DF00001F0F350F4100DE0FC0EDBCFE6FFFD0E2A
:100E0000DBCFE6FFF5DDE552E552DF6EDF5001E1B5
:100E100069D7DF50E552E552E552E5CFDAFFE7CF7B
:100E2000D9FF1200D9CFE6FFDACFE6FFE1CFD9FF35
:100E3000E2CFDAFF090EE12402E3E168E652E16E57
:100E4000FC0EDBCFE9FFFD0EDBCFEAFF020EE92649
:100E5000000EEA22050EEECFDBFF060EEDCFDBFF24
:100E60000B0EE66EE66A200EE66EE66A050EDBCF36
:100E7000E6FF060EDBCFE6FF1CEC00F0006E060E70
:100E8000E15C02E2E16AE552E16E0050040EDB6AC9
:100E9000030EDB6A080EF36E020EF3CFDBFFFA0ED1
:100EA000DBCFE9FFFB0EDBCFEAFF070EEECFDBFF68
:100EB000080EEDCFDBFF030EDBCFF3FFDB2AF35091
:100EC000E76E070EDBCFE9FF080EDBCFEAFFE75046
:100ED000E926000EEA22EFCFDFFFDF5020083CE2D8
:100EE0002F0EDF5C39E02E0EDF5C09E0020EDB50D6
:100EF000F36E040EDBCFF4FFF350F45C12E3020E4A
:100F0000DB50080829E12E0EDF5C26E1080EF36EA7
:100F1000040EF3CFDBFF0B0EF36E020EF3CFDBFFFD
:100F2000CAD7610EDF5C05E3DF507A0802E3200ECA
:100F3000DF5E040EDBCFF3FFDB2AF350E76E050E16
:100F4000DBCFE9FF060EDBCFEAFFE750E926000E14
:100F5000EA22DFCFEFFFAFD7030EDB50E76E070EBD
:100F6000DBCF00F0080EDBCF01F0E7500026000ECB
:100F70000122FA0EDBCFE9FFFB0EDBCFEAFF00C058
:100F8000EEFF01C0EDFFDF50200802E3010E01D0AB
:100F9000000EE66E0B0EE76E050EDBCFE9FF060EC8
:100FA000DBCFEAFFE750E926000EEA22E552E750E0
:100FB000EF6E000E006E090EE15C02E2E16AE5529E
:100FC000E16E0050E552E5CFDAFFE7CFD9FF12001E
:100FD000D9CFE6FFDACFE6FFE1CFD9FFE2CFDAFFE4
:100FE000E652F80EDBCFE9FFF90EDBCFEAFFEF5058
:100FF000200806E1F80EDB2AF90EF3E3DB2AF1D72D
:10100000F80EDBCFE9FFF90EDBCFEAFFEF502F0838
:1010100005E1F80EDB2AF90E01E3DB2AFC0EDBCF3B
:10102000E9FFFD0EDBCFEAFF040EE926000EEA22FF
:10103000EE6AEE6AEE6AEE6AF80EDBCFE9FFF90EB1
:10104000DBCFEAFFEF50200813E3FC0EDBCFE6FF17
:10105000FD0EDBCFE6FFF8EC03F0E552E552DF6E64
:10106000FA0EDBCFE9FFFB0EDBCFEAFFEF6AE0D041
:10107000D950F80FE66EFF0EDA20E66EFC0EDBCFDD
:10108000E6FFFD0EDBCFE6FFCDDEE552E552E55291
:10109000E552DF6EDF5001E0CBD0FA0EDBCFE6FF8A
:1010A000FB0EDBCFE6FFFC0EDBCFE6FFFD0EDBCF5A
:1010B000E6FF00DEE552E552E552E552DF6EDF5015
:1010C0001AE0030EDF5C01E0B3D0FC0EDBCFE9FFDA
:1010D000FD0EDBCFEAFF020EE926000EEA22EE50FB
:1010E000EFCFEAFFE96E0B0EE926000EEA22EF5081
:1010F00001E09ED024D0FC0EDBCFE9FFFD0EDBCF5C
:10110000EAFF020EE926000EEA22EE50EFCFEAFFD8
:10111000E96E0B0EE926000EEA22EF5001E088D0BE
:101120000B0EE76EFA0EDBCFE9FFFB0EDBCFEAFF1B
:10113000E750E926000EEA22EF50100B03E1040EFF
:10114000DF6E76D0140EE76EFA0EDBCFE9FFFB0EF2
:10115000DBCFEAFFE750E926000EEA22010EE9267E
:10116000000EEA22EFCF04F004C005F0046A140E6A
:10117000E76EFA0EDBCFE9FFFB0EDBCFEAFFE750AD
:10118000E926000EEA22EF500410006E05C001F0BF
:10119000026A036A100E1F0B07E0D8900036013672
:1011A00002360336E806F9E11A0EE76EFA0EDBCFD7
:1011B000E9FFFB0EDBCFEAFFE750E926000EEA224B
:1011C000010EE926000EEA22EFCF0AF00AC00BF06A
:1011D0000A6A1A0EE76EFA0EDBCFE9FFFB0EDBCFD1
:1011E000EAFFE750E926000EEA22EF5000010A105C
:1011F000066E0BC007F0086A096AE85000120B502F
:1012000001120850021209500312FC0EDBCFE9FF55
:10121000FD0EDBCFEAFF040EE926000EEA2200C035
:10122000EEFF01C0EEFF02C0EEFF03C0EEFF20D7CD
:10123000DF50E552E552E5CFDAFFE7CFD9FF1200E4
:10124000D9CFE6FFDACFE6FFE1CFD9FFE2CFDAFF71
:10125000020EE66EE66AFE0EE66E010EE66ED950EE
:10126000F80FE96EFF0EDA20EA6EEECFE6FFEECF62
:10127000E6FFEECFE6FFEFCFE6FFFC0EDBCFE6FFAB
:10128000FD0EDBCFE6FF0AEC42F0006E0A0EE15CD9
:1012900002E2E16AE552E16E0050000902E0030E4D
:1012A000BAD0010EE76EFC0EDBCFE9FFFD0EDBCFFF
:1012B000EAFFE750E926000EEA22EFCF02F002C073
:1012C00003F0026AFC0EDBCFE9FFFD0EDBCFEAFF85
:1012D000EF5000010210006E03C001F0550E00181F
:1012E00002E1AA0E011802E0020E95D0020EE66E8F
:1012F000E66A360EE66EE66AD950F80FE96EFF0E22
:10130000DA20EA6EEECFE6FFEECFE6FFEECFE6FFA5
:10131000EFCFE6FFFC0EDBCFE6FFFD0EDBCFE6FFF7
:101320000AEC42F0006E0A0EE15C02E2E16AE5526C
:10133000E16E0050000923E1010EE76EFC0EDBCFE9
:10134000E9FFFD0EDBCFEAFFE750E926000EEA22B7
:10135000EFCF03F003C004F0036AFC0EDBCFE9FF1C
:10136000FD0EDBCFEAFFEF5000010310016E04C059
:1013700002F0460E011803E1410E021849E0020E88
:10138000E66EE66A520EE66EE66AD950F80FE96E2E
:10139000FF0EDA20EA6EEECFE6FFEECFE6FFEECFED
:1013A000E6FFEFCFE6FFFC0EDBCFE6FFFD0EDBCF67
:1013B000E6FF0AEC42F0006E0A0EE15C02E2E16A2E
:1013C000E552E16E0050000925E1010EE76EFC0ECA
:1013D000DBCFE9FFFD0EDBCFEAFFE750E926000E89
:1013E000EA22EFCF03F003C004F0036AFC0EDBCF68
:1013F000E9FFFD0EDBCFEAFFEF5000010310016EA5
:1014000004C002F0460E011805E1410E021802E187
:10141000000E01D0010EE552E5CFDAFFE7CFD9FF8C
:101420001200D9CFE6FFDACFE6FFE1CFD9FFE2CF56
:10143000DAFF350EE12402E3E168E652E16E0401D1
:10144000FE6BFF6BD950FC0FE96EFF0EDA20EA6EDF
:10145000EE50ED1002E10EEF0FF09FEC40F0010BAB
:1014600003E0020E0FEF0FF0250EDB6A260EDB6A9B
:10147000270EDB6A280EDB6AD950250FE96E000EB5
:10148000DA20EA6EEECFE6FFEECFE6FFEECFE6FF24
:10149000EFCFE6FFD950010FE66E000EDA20E66EC0
:1014A000CFDE006E060EE15C02E2E16AE552E16E1B
:1014B0000050DF6EDF0401E09CD0100EE66EE66A9D
:1014C000BE0EE66E010EE66ED950250FE96E000ED7
:1014D000DA20EA6EEECFE6FFEECFE6FFEECFE6FFD4
:1014E000EFCFE6FFD950010FE66E000EDA20E66E70
:1014F0000AEC42F0006E0A0EE15C02E2E16AE5529B
:10150000E16E0050000902E0030E72D0050EDB50C0
:1015100070E00C0EDBCF00F0016A026A036A180E5D
:101520001F0B07E0D8900036013602360336E80676
:10153000F9E10B0EDBCF04F0056A066A076A100EAC
:101540001F0B07E0D8900436053606360736E80646
:10155000F9E1045000120550011206500212075022
:1015600003120A0EDBCF08F008C009F0086A0A6A05
:101570000B6A08500012095001120A5002120B5057
:101580000312090EDBCF0CF00D6A0E6A0F6A0C50C5
:1015900000120D5001120E5002120F500312250EB0
:1015A00000C0DBFF260E01C0DBFF270E02C0DBFF01
:1015B000280E03C0DBFFD950250FE96E000EDA209C
:1015C000EA6EEECFE6FFEECFE6FFEECFE6FFEFCF1F
:1015D000E6FFD950010FE66E000EDA20E66E30DE2F
:1015E000006E060EE15C02E2E16AE552E16E005037
:1015F000DF6E030EDF5C2BE0DF5003E0070E0FEF22
:101600000FF0240EE66EE66A0D0EE66EE66AD9501D
:10161000250FE96E000EDA20EA6EEECFE6FFEECF80
:10162000E6FFEECFE6FFEFCFE6FFD950010FE66E03
:10163000000EDA20E66E0AEC42F0006E0A0EE15C63
:1016400002E2E16AE552E16E0050000902E0010E9B
:10165000E6D3D950170FE96E000EDA20EA6E0D0EB0
:10166000E95E000EEA5A010EE926000EEA22EFCFEB
:1016700002F002C003F0026AD950170FE96E000EA3
:10168000DA20EA6E0D0EE95E000EEA5AEF50000114
:101690000210006E290E00C0DBFF2A0E03C0DBFF24
:1016A0002B0EDB6A2C0EDB6A290EDBCF00F02A0E34
:1016B000DBCF01F02B0EDBCF02F02C0EDBCF03F0E3
:1016C000005001100210031001E082D0D950250F04
:1016D000E96E000EDA20EA6E0D0EE95E000EEA5A9F
:1016E000030EE926000EEA22EFCF00F0016A026A3B
:1016F000036A180E1F0B07E0D89000360136023639
:101700000336E806F9E1D950250FE96E000EDA201C
:10171000EA6E0D0EE95E000EEA5A020EE926000E90
:10172000EA22EFCF04F0056A066A076A100E1F0B63
:1017300007E0D8900436053606360736E806F9E1A4
:1017400004500012055001120650021207500312F5
:10175000D950250FE96E000EDA20EA6E0D0EE95E13
:10176000000EEA5A010EE926000EEA22EFCF08F039
:1017700008C009F0086A0A6A0B6A0850001209508A
:1017800001120A5002120B500312D950250FE96EB4
:10179000000EDA20EA6E0D0EE95E000EEA5AEFCF77
:1017A0000CF00D6A0E6A0F6A0C5000120D500112F7
:1017B0000E5002120F500312290E00C0DBFF2A0E3A
:1017C00001C0DBFF2B0E02C0DBFF2C0E03C0DBFFD2
:1017D000040EDBCF00F0016A026A036AD950290FB8
:1017E000E96E000EDA20EA6E00C042F001C043F05C
:1017F00002C044F003C045F0EECF3DF0EECF3EF026
:10180000EECF3FF0EFCF40F085EC4BF03CC0EDFF6A
:101810003BC0EDFF3AC0EDFF39C0EFFFD9500F0FCD
:10182000E96E000EDA20EA6E0D0EE95E000EEA5A4D
:10183000010EE926000EEA22EFCF04F004C005F005
:10184000046AD9500F0FE96E000EDA20EA6E0D0E11
:10185000E95E000EEA5AEF500410006E05C001F078
:10186000026A036AD950250FE96E000EDA20EA6E8B
:10187000EE500026EE500122EE500222EE500322DE
:10188000FC0EDBCFE9FFFD0EDBCFEAFF0A0EE926F7
:10189000000EEA2200C0EEFF01C0EEFF02C0EEFF24
:1018A00003C0EEFFFC0EDBCFE9FFFD0EDBCFEAFF4E
:1018B000020EE926000EEA22010EDBCFEFFFD9501F
:1018C000120FE96E000EDA20EA6E0D0EE95E000ED0
:1018D000EA5A010EE926000EEA22EFCF02F002C01A
:1018E00003F0026AD950120FE96E000EDA20EA6E98
:1018F0000D0EE95E000EEA5AEF500210006E03C0B2
:1019000001F0FC0EDBCFE9FFFD0EDBCFEAFF040E9A
:10191000E926000EEA2200C0EEFF01C0EDFFD9501B
:10192000140FE96E000EDA20EA6E0D0EE95E000E6D
:10193000EA5A010EE926000EEA22EFCF02F002C0B9
:1019400003F0026AD950140FE96E000EDA20EA6E35
:101950000D0EE95E000EEA5AEF500210006E2D0ED9
:1019600000C0DBFF2E0E03C0DBFF2F0EDB6A300E44
:10197000DB6A2D0EDBCF00F02E0EDBCF01F02F0E39
:10198000DBCF02F0300EDBCF03F00050011002106D
:10199000031001E082D0D950210FE96E000EDA2049
:1019A000EA6E0D0EE95E000EEA5A030EE926000EFD
:1019B000EA22EFCF00F0016A026A036A180E1F0BD9
:1019C00007E0D8900036013602360336E806F9E122
:1019D000D950210FE96E000EDA20EA6E0D0EE95E95
:1019E000000EEA5A020EE926000EEA22EFCF04F0BA
:1019F000056A066A076A100E1F0B07E0D8900436C6
:101A0000053606360736E806F9E10450001205509F
:101A100001120650021207500312D950210FE96E2D
:101A2000000EDA20EA6E0D0EE95E000EEA5A010E93
:101A3000E926000EEA22EFCF08F008C009F0086A94
:101A40000A6A0B6A08500012095001120A50021269
:101A50000B500312D950210FE96E000EDA20EA6E06
:101A60000D0EE95E000EEA5AEFCF0CF00D6A0E6A19
:101A70000F6A0C5000120D5001120E5002120F503E
:101A800003122D0E00C0DBFF2E0E01C0DBFF2F0E58
:101A900002C0DBFF300E03C0DBFFFC0EDBCFE9FF33
:101AA000FD0EDBCFEAFF020EE926000EEA22EFCFA1
:101AB0001AF01B6A1C6A1D6AD9500F0FE96E000EDE
:101AC000DA20EA6E0D0EE95E000EEA5A010EE926F2
:101AD000000EEA22EFCF14F014C015F0146AD950AA
:101AE0000F0FE96E000EDA20EA6E0D0EE95E000EB1
:101AF000EA5AEF5000011410106E15C011F0126A6E
:101B0000136AD9502D0FE96E000EDA20EA6E1050DC
:101B1000EE5C0C6E1550EE580D6E1250EE580E6EB7
:101B20001350EE580F6ED950290FE96E000EDA20CF
:101B3000EA6EEE500C5C086EEE500D58096EEE50D9
:101B40000E580A6EEE500F580B6EFC0EDBCFE9FFFD
:101B5000FD0EDBCFEAFF040EE926000EEA22EECFEF
:101B600016F0EFCF17F0040E0F0B05E0D8901732E8
:101B70001632E806FBE1186A196A1650085C046E12
:101B800017500958056E18500A58066E19500B5810
:101B9000076E04C03DF005C03EF006C03FF0406E49
:101BA0001AC042F01BC043F01CC044F01DC045F0F9
:101BB000EAEC4BF03DC000F03EC001F03FC002F047
:101BC00040C003F0020E0026000E01220222032272
:101BD000310E00C0DBFF320E01C0DBFF330E02C04E
:101BE000DBFF340E03C0DBFFFC0EDBCFE9FFFD0E95
:101BF000DBCFEAFF060EE926000EEA22310EDBCF2C
:101C0000EEFF320EDBCFEEFF330EDBCFEEFF340EF6
:101C1000DBCFEEFF020EDF6ED950310FE96E000E02
:101C2000DA20EA6EF70EEE5C0F0EEE58000EEE585C
:101C3000000EEE5802E2010EDF6ED950310FE96E50
:101C4000000EDA20EA6EF70EEE5CFF0EEE58000E84
:101C5000EE58000EEE5802E3030EDF6EFC0EDBCFF3
:101C6000E9FFFD0EDBCFEAFFDFCFEFFF030EDF5C06
:101C700047E1230EDBCF00F0016A026A036A180E07
:101C80001F0B07E0D8900036013602360336E8060F
:101C9000F9E1220EDBCF04F0056A066A076A100E2E
:101CA0001F0B07E0D8900436053606360736E806DF
:101CB000F9E10450001205500112065002120750BB
:101CC0000312210EDBCF08F008C009F0086A0A6A87
:101CD0000B6A08500012095001120A5002120B50F0
:101CE0000312200EDBCF0CF00D6A0E6A0F6A0C5047
:101CF00000120D5001120E5002120F5003121ED08E
:101D0000290EDBCF00F02A0EDBCF01F02B0EDBCF4C
:101D100002F02C0EDBCF03F0FC0EDBCFE9FFFD0E53
:101D2000DBCFEAFF0A0EE926000EEA22EE5000267B
:101D3000EE500122EE500222EE500322FC0EDBCFC9
:101D4000E9FFFD0EDBCFEAFF0E0EE926000EEA22C8
:101D500000C0EEFF01C0EEFF02C0EEFF03C0EEFFC9
:101D6000290EDBCF00F02A0EDBCF01F02B0EDBCFEC
:101D700002F02C0EDBCF03F0FC0EDBCFE9FFFD0EF3
:101D8000DBCFEAFF0A0EE926000EEA22EE5000261B
:101D9000EE500122EE500222EE500322FC0EDBCF69
:101DA000E9FFFD0EDBCFEAFF040EE926000EEA2272
:101DB000EECF04F0EFCF05F0040E0F0B05E0D89046
:101DC00005320432E806FBE1066A076A0450002681
:101DD000055001220650022207500322FC0EDBCFE1
:101DE000E9FFFD0EDBCFEAFF120EE926000EEA2224
:101DF00000C0EEFF01C0EEFF02C0EEFF03C0EEFF29
:101E0000FC0EDBCFE9FFFD0EDBCFEAFFEE52EF6AFF
:101E1000FC0EDBCFFEF4FD0EDBCFFFF4000E006EF8
:101E2000350EE15C02E2E16AE552E16E0050E552F6
:101E3000E5CFDAFFE7CFD9FF1200D9CFE6FFDACF3F
:101E4000E6FFE1CFD9FFE2CFDAFF3F0EE12402E364
:101E5000E168E652E16E3D0EFEC4DBFF3E0EFFC4BC
:101E6000DBFFD9503D0FE96E000EDA20EA6EEE502E
:101E7000ED1002E1060EEBD03D0EDBCFE9FF3E0E8A
:101E8000DBCFEAFFEE52EF6AD950110F006E000E61
:101E9000DA20016E030E00C0DBFF040E01C0DBFF81
:101EA000FC0EDBCFE6FFFD0EDBCFE6FFD9501D0FAA
:101EB000E66E000EDA20E66ED950010FE66E000ED7
:101EC000DA20E66EE8EC07F0006E060EE15C02E256
:101ED000E16AE552E16E0050DF6EDF5002E0DF5054
:101EE000B6D01D0EDB5004E0280EDB50100B02E0D4
:101EF000030EADD0320EDBCF04F004C005F0046A4F
:101F0000310EDB500410006E05C001F0026A036A56
:101F1000100E1F0B07E0D89000360136023603364C
:101F2000E806F9E1380EDBCF0AF00AC00BF00A6AC6
:101F3000370EDB500A10086A096AE85000120B508D
:101F4000011208500212095003123D0EDBCFE9FFC7
:101F50003E0EDBCFEAFF1E0EE926000EEA2200C08D
:101F6000EEFF01C0EEFF02C0EEFF03C0EEFF3C0E2D
:101F7000DBCF00F0016A026A036A180E1F0B07E04C
:101F8000D8900036013602360336E806F9E13B0EFA
:101F9000DBCF04F0056A066A076A100E1F0B07E024
:101FA000D8900436053606360736E806F9E10450BF
:101FB00000120550011206500212075003123A0E89
:101FC000DBCF08F008C009F0086A0A6A0B6A0850FB
:101FD0000012095001120A5002120B500312390E5E
:101FE000DBCF0CF00D6A0E6A0F6A0C5000120D5018
:101FF00001120E5002120F5003123D0EDBCFE9FF0B
:102000003E0EDBCFEAFF1A0EE926000EEA2200C0E0
:10201000EEFF01C0EEFF02C0EEFF03C0EEFF3D0E7B
:10202000DBCFE9FF3E0EDBCFEAFF160EE926000EFE
:10203000EA22EE6AEE6AEE6AEE6A3D0EDBCFE9FF57
:102040003E0EDBCFEAFFEE52010EEF6E000E006E89
:102050003F0EE15C02E2E16AE552E16E0050E552BA
:10206000E5CFDAFFE7CFD9FF1200D9CFE6FFDACF0D
:10207000E6FFE1CFD9FFE2CFDAFF140EE12402E35D
:10208000E168E652E16EFC0EDBCF3FF0FD0EDBCFE8
:1020900040F0100E3FC0DBFF110E40C0DBFF120E00
:1020A000FEC4DBFF130EFFC4DBFFF80EDBCFE9FF3E
:1020B000F90EDBCFEAFFEE6AED6AD950120FE96E36
:1020C000000EDA20EA6EEE50ED1002E1060E87D225
:1020D000120EDBCFE9FF130EDBCFEAFFEE52EF501B
:1020E000010B02E1050E7BD2120EDBCFE9FF130ECE
:1020F000DBCFEAFF1A0EE926000EEA22EECF04F04B
:10210000EECF05F0EECF06F0EFCF07F0120EDBCFEB
:10211000E9FF130EDBCFEAFF160EE926000EEA22D6
:10212000EE50045C006EEE500558016EEE500658FD
:10213000026EEE500758036E090E00C0DBFF0A0E58
:1021400001C0DBFF0B0E02C0DBFF0C0E03C0DBFF88
:10215000FA0EDBCF00F0FB0EDBCF01F0026A036A60
:10216000D950090FE96E000EDA20EA6E0050EE5CDD
:102170000150EE580250EE580350EE580CE2090E92
:10218000DBCF3FF00A0EDBCF40F0FA0E3FC0DBFFA3
:10219000FB0E40C0DBFFD950FA0FE96EFF0EDA20CC
:1021A000EA6EEE50ED1001E10FD2120EDBCFE9FF27
:1021B000130EDBCFEAFF160EE926000EEA22EECF61
:1021C00000F0EECF01F0010E0116026A036A005022
:1021D00001100210031001E010D1120EDBCFE9FF55
:1021E000130EDBCFEAFF160EE926000EEA22EECF31
:1021F00000F0EECF01F0EECF02F0EFCF03F0090ECA
:10220000D8900332023201320032E806F9E1120EB0
:10221000DBCFE9FF130EDBCFEAFF020EE926000E4B
:10222000EA22EF04046E056A066A076AE85000169F
:102230000550011606500216075003160F0E00C077
:10224000DBFFDB5001E07DD0120EDBCFE9FF130E88
:10225000DBCFEAFF160EE926000EEA22EECF04F0ED
:10226000EECF05F0EECF06F0EFCF07F004500510EB
:102270000610071013E1120EDBCFE9FF130EDBCFC0
:10228000EAFF1E0EE926000EEA22EECF00F0EECFA6
:1022900001F0EECF02F0EFCF03F020D0120EDBCF33
:1022A000E9FF130EDBCFEAFF220EE926000EEA2239
:1022B000EECFE6FFEECFE6FFEECFE6FFEFCFE6FF95
:1022C000B2EC00F0E552E552E552E5523DC000F0B7
:1022D0003EC001F03FC002F040C003F0010E00C05C
:1022E000DBFF020E01C0DBFF030E02C0DBFF040EAA
:1022F00003C0DBFFD950010FE96E000EDA20EA6E51
:10230000D880010EEE54000EEE54000EEE54000E76
:10231000EE5401E35BD1120EDBCFE9FF130EDBCFEE
:10232000EAFF220EE926000EEA22010EDBCFEEFFC5
:10233000020EDBCFEEFF030EDBCFEEFF040EDBCF92
:10234000EEFF120EDBCFE9FF130EDBCFEAFF220E0A
:10235000E926000EEA22EECFE6FFEECFE6FFEECF53
:10236000E6FFEFCFE6FF66EC03F0E552E552E552FB
:10237000E552050E3DC0DBFF060E3EC0DBFF070E3B
:102380003FC0DBFF080E40C0DBFF050EDBCF00F0D7
:10239000060EDBCF01F0070EDBCF02F0080EDBCF1D
:1023A00003F0005001100210031001E10FD10F0ED5
:1023B000DBCF00F0016A026A036AD950050FE96EAB
:1023C000000EDA20EA6EEE500026EE500122EE50AA
:1023D0000222EE500322120EDBCFE9FF130EDBCFF9
:1023E000EAFF260EE926000EEA2200C0EEFF01C039
:1023F000EEFF02C0EEFF03C0EEFF046A020E056EA0
:10240000066A076A120EDBCFE9FF130EDBCFEAFF85
:10241000160EE926000EEA22EECF3DF0EECF3EF09A
:10242000EECF3FF0EFCF40F0426A020E436E446AB7
:10243000456AEAEC4BF03950045C006E3A5005589E
:10244000016E3B5006583C5007580D0E00C0DBFF94
:102450000E0E01C0DBFF0D0EDBCF00F00E0EDBCF4A
:1024600001F0FA0EDBCF02F0FB0EDBCF03F00050E1
:10247000025C015003580CE2FA0EDBCF3FF0FB0E7A
:10248000DBCF40F00D0E3FC0DBFF0E0E40C0DBFF88
:102490000D0EDBCFE6FF0E0EDBCFE6FF120EDBCF1D
:1024A000E9FF130EDBCFEAFF160EE926000EEA2243
:1024B000EECF00F0EECF01F0010E0116026A036AC2
:1024C00000C0E6FF01C0E6FF120EDBCFE9FF130EEE
:1024D000DBCFEAFF260EE926000EEA22EECFE6FF6A
:1024E000EECFE6FFEECFE6FFEFCFE6FFD950FC0FD1
:1024F000E96EFF0EDA20EA6EEE50ED1003E1046A99
:10250000056A06D0100EDBCF04F0110EDBCF05F00C
:1025100004C0E6FF05C0E6FF0AEC42F0066E0A0EB4
:10252000E15C02E2E16AE552E16E0650DF6EDF50E7
:102530004DE10D0EDBCF00F00E0EDBCF01F0026A95
:10254000036A120EDBCFE9FF130EDBCFEAFF160E94
:10255000E926000EEA220050EE260150EE2202503B
:10256000EE220350EE220D0EDBCF00F00E0EDBCF7D
:1025700001F0D950100FE96E000EDA20EA6E00501B
:10258000EE260150ED220D0EDBCF00F00E0EDBCF5C
:1025900001F0D950FA0FE96EFF0EDA20EA6E005012
:1025A000EE5E0150ED5A0D0EDBCF00F00E0EDBCFCC
:1025B00001F0F80EDBCFE9FFF90EDBCFEAFF0050A8
:1025C000EE260150ED22E7D5000E09D0120EDBCF2A
:1025D000E9FF130EDBCFEAFFEE52EF6A010E006E49
:1025E000140EE15C02E2E16AE552E16E0050E55250
:1025F000E5CFDAFFE7CFD9FF1200D9CFE6FFDACF78
:10260000E6FFE1CFD9FFE2CFDAFF130EE12402E3C8
:10261000E168E652E16EFC0EDBCF3FF0FD0EDBCF52
:1026200040F00C0E3FC0DBFF0D0E40C0DBFF110E73
:10263000FEC4DBFF120EFFC4DBFFF80EDBCFE9FFA9
:10264000F90EDBCFEAFFEE6AED6AD950110FE96EA1
:10265000000EDA20EA6EEE50ED1002E1060EDFD237
:10266000110EDBCFE9FF120EDBCFEAFFEE52EF5087
:10267000010B02E1050ED3D2D950FA0FE96EFF0E1D
:10268000DA20EA6EEE50ED1027E1110EDBCFE9FF04
:10269000120EDBCFEAFFEE52EF50400B14E0E66A79
:1026A000E66AE66AE66A000EE66EE66ADBEC42F08F
:1026B000006E060EE15C02E2E16AE552E16E005056
:1026C000000901E0A3D2110EDBCFE9FF120EDBCF30
:1026D000EAFFEE52EF9C98D2110EDBCFE9FF120E0B
:1026E000DBCFEAFFEE52EF50400B0CE1110EDBCFD7
:1026F000E9FF120EDBCFEAFF160EE926000EEA22F2
:10270000EE6AEE90110EDBCFE9FF120EDBCFEAFF8F
:102710001A0EE926000EEA22EECF04F0EECF05F005
:10272000EECF06F0EFCF07F0110EDBCFE9FF120E70
:10273000DBCFEAFF160EE926000EEA22EE50045C1B
:10274000006EEE500558016EEE500658026EEE50C7
:102750000758036E080E00C0DBFF090E01C0DBFF47
:102760000A0E02C0DBFF0B0E03C0DBFFFA0EDBCF4D
:1027700000F0FB0EDBCF01F0026A036AD950080FAC
:10278000E96E000EDA20EA6E0050EE5C0150EE5861
:102790000250EE580350EE580CE2080EDBCF3FF02B
:1027A000090EDBCF40F0FA0E3FC0DBFFFB0E40C04E
:1027B000DBFFD950FA0FE96EFF0EDA20EA6EEE5019
:1027C000ED1001E121D2110EDBCFE9FF120EDBCFBC
:1027D000EAFF160EE926000EEA22EECF00F0EFCF58
:1027E00001F00001010E01160050011001E035D189
:1027F000110EDBCFE9FF120EDBCFEAFF160EE92642
:10280000000EEA22EECF00F0EECF01F0EECF02F0A4
:10281000EFCF03F0090ED8900332023201320032BA
:10282000E806F9E1110EDBCFE9FF120EDBCFEAFF7C
:10283000020EE926000EEA22EF04046E056A066A1B
:10284000076AE85000160550011606500216075098
:1028500003160E0E00C0DBFFDB5001E079D0110E35
:10286000DBCFE9FF120EDBCFEAFF160EE926000EE2
:10287000EA22EECF04F0EECF05F0EECF06F0EFCF78
:1028800007F0045005100610071013E1110EDBCFFE
:10289000E9FF120EDBCFEAFF1E0EE926000EEA2248
:1028A000EECF00F0EECF01F0EECF02F0EFCF03F06D
:1028B00020D0110EDBCFE9FF120EDBCFEAFF220E94
:1028C000E926000EEA22EECFE6FFEECFE6FFEECFDE
:1028D000E6FFEFCFE6FFB2EC00F0E552E552E5523D
:1028E000E5523DC000F03EC001F03FC002F040C0E4
:1028F00003F000C0DFFF010E01C0DBFF020E02C0CB
:10290000DBFF030E03C0DBFFD9CFE9FFDACFEAFF1D
:10291000D880010EEE54000EEE54000EEE54000E60
:10292000EE5401E373D1110EDBCFE9FF120EDBCFC2
:10293000EAFF220EE926000EEA22DFCFEEFF010EAB
:10294000DBCFEEFF020EDBCFEEFF030EDBCFEEFFA1
:10295000110EDBCFE9FF120EDBCFEAFF220EE926D4
:10296000000EEA22EECFE6FFEECFE6FFEECFE6FF67
:10297000EFCFE6FF66EC03F0E552E552E552E55293
:10298000040E3DC0DBFF050E3EC0DBFF060E3FC060
:10299000DBFF070E40C0DBFF040EDBCF00F0050EAF
:1029A000DBCF01F0060EDBCF02F0070EDBCF03F02A
:1029B000005001100210031001E128D10E0EDBCFF0
:1029C00000F0016A026A036AD950040FE96E000E32
:1029D000DA20EA6EEE500026EE500122EE5002227E
:1029E000EE500322110EDBCFE9FF120EDBCFEAFF20
:1029F000260EE926000EEA2200C0EEFF01C0EEFF1F
:102A000002C0EEFF03C0EEFF110EDBCFE9FF120E96
:102A1000DBCFEAFF260EE926000EEA22EECFE6FF24
:102A2000EECFE6FFEECFE6FFEFCFE6FFE66EE66A1B
:102A3000DBEC42F0006E060EE15C02E2E16AE55278
:102A4000E16E0050000901E0E1D0110EDBCFE9FF9B
:102A5000120EDBCFEAFFEE52EF8C110EDBCFE9FF57
:102A6000120EDBCFEAFF160EE926000EEA22EECFA9
:102A700000F0EFCF01F00001010E0116000ED8802A
:102A80000056020E01560F0E00C0DBFF100E01C0F3
:102A9000DBFF0F0EDBCF00F0100EDBCF01F0FA0EE4
:102AA000DBCF02F0FB0EDBCF03F00050025C0150E5
:102AB00003580CE2FA0EDBCF3FF0FB0EDBCF40F009
:102AC0000F0E3FC0DBFF100E40C0DBFF0F0EDBCF51
:102AD00000F0100EDBCF01F0026A036A00C0E6FFCF
:102AE00001C0E6FF02C0E6FF03C0E6FF0C0EDBCF2D
:102AF000E6FF0D0EDBCFE6FFDBEC42F0046E060EC8
:102B0000E15C02E2E16AE552E16E0450000901E095
:102B10007DD00F0EDBCF00F0100EDBCF01F0026A8C
:102B2000036A110EDBCFE9FF120EDBCFEAFF160EB0
:102B3000E926000EEA220050EE260150EE22025055
:102B4000EE220350EE220F0EDBCF00F0100EDBCF93
:102B500001F0D9500C0FE96E000EDA20EA6E005039
:102B6000EE260150ED220F0EDBCF00F0100EDBCF72
:102B700001F0D950FA0FE96EFF0EDA20EA6E00502C
:102B8000EE5E0150ED5A0F0EDBCF00F0100EDBCFE2
:102B900001F0F80EDBCFE9FFF90EDBCFEAFF0050C2
:102BA000EE260150ED22110EDBCFE9FF120EDBCF36
:102BB000EAFF160EE926000EEA22EECF00F0EFCF74
:102BC00001F00001010E01160050011001E0F1D5E5
:102BD000E66AE66AE66AE66A000EE66EE66ADBEC3C
:102BE00042F0006E060EE15C02E2E16AE552E16E3F
:102BF000005000090BE1110EDBCFE9FF120EDBCF15
:102C0000EAFFEE52EF9CD5D5000E09D0110EDBCFB6
:102C1000E9FF120EDBCFEAFFEE52EF6A010E006E03
:102C2000130EE15C02E2E16AE552E16E0050E5520A
:102C3000E5CFDAFFE7CFD9FF1200D9CFE6FFDACF31
:102C4000E6FFE1CFD9FFE2CFDAFF120EE12402E383
:102C5000E168E652E16E100EFEC4DBFF110EFFC408
:102C6000DBFFD950100FE96E000EDA20EA6EEE504D
:102C7000ED1002E1060EEDD2100EDBCFE9FF110ED2
:102C8000DBCFEAFFEE52EF50010B02E1050EE1D27D
:102C9000FA0EDBCF00F0FB0EDBCF01F0FC0EDBCF3A
:102CA00002F0FD0EDBCF03F0100EDBCFE9FF110EBB
:102CB000DBCFEAFF1A0EE926000EEA220050EE5C96
:102CC0000150EE580250EE580350EE5816E2100E26
:102CD000DBCFE9FF110EDBCFEAFF1A0EE926000E6B
:102CE000EA22FA0EEECFDBFFFB0EEECFDBFFFC0E8F
:102CF000EECFDBFFFD0EEECFDBFF100EDBCFE9FFEB
:102D0000110EDBCFEAFF160EE926000EEA220C0EAA
:102D1000EECFDBFF0D0EEECFDBFF0E0EEECFDBFFB7
:102D20000F0EEECFDBFF100EDBCFE9FF110EDBCF76
:102D3000EAFF160EE926000EEA22EE6AEE6AEE6A55
:102D4000EE6AD950FA0FE96EFF0EDA20EA6ED880EB
:102D5000000EEE54000EEE54000EEE54000EEE5433
:102D600001E36CD2100EDBCFE9FF110EDBCFEAFFDF
:102D7000020EE926000EEA22EFCF3DF03E6A3F6ADE
:102D8000406A426A020E436E446A456A85EC4BF023
:102D9000040E39C0DBFF050E3AC0DBFF060E3BC058
:102DA000DBFF070E3CC0DBFFD9500C0FE96E000EB5
:102DB000DA20EA6ED880000EEE54000EEE54000EBB
:102DC000EE54000EEE5401E3D5D00C0EDBCF08F02C
:102DD0000D0EDBCF09F00E0EDBCF0AF00F0EDBCFAE
:102DE0000BF00806000E095A0A5A0B5A08C03DF0AB
:102DF00009C03EF00AC03FF00BC040F0040EDBCF2C
:102E000042F0050EDBCF43F0060EDBCF44F0070E99
:102E1000DBCF45F0EAEC4BF03DC004F03EC005F0DE
:102E20003FC006F040C007F0FA0EDBCF00F0FB0E0B
:102E3000DBCF01F0FC0EDBCF02F0FD0EDBCF03F0A9
:102E40000006000E015A025A035A00C03DF001C0AC
:102E50003EF002C03FF003C040F0040EDBCF42F072
:102E6000050EDBCF43F0060EDBCF44F0070EDBCFC1
:102E700045F0EAEC4BF004503D5C05503E580650DE
:102E80003F580750405876E30C0EDBCF00F00D0E94
:102E9000DBCF01F00E0EDBCF02F00F0EDBCF03F025
:102EA0000006000E015A025A035A040EDBCF04F04A
:102EB000050EDBCF05F0060EDBCF06F0070EDBCFED
:102EC00007F00406000E055A065A075A041E051E8E
:102ED000061E071E04500016055001160650021665
:102EE00007500316100EDBCFE9FF110EDBCFEAFF10
:102EF000160EE926000EEA2200C0EEFF01C0EEFF2A
:102F000002C0EEFF03C0EEFF100EDBCFE9FF110E93
:102F1000DBCFEAFF160EE926000EEA22EECF00F024
:102F2000EECF01F0EECF02F0EFCF03F0D950FA0F61
:102F3000E96EFF0EDA20EA6E0050EE5E0150EE5AA6
:102F40000250EE5A0350EE5A100EDBCFE9FF110E7D
:102F5000DBCFEAFF220EE926000EEA22EECFDFFFEA
:102F6000010EEECFDBFF020EEECFDBFF030EEECF46
:102F7000DBFF2AD0100EDBCFE9FF110EDBCFEAFF1B
:102F80001E0EE926000EEA22EECFDFFF010EEECF85
:102F9000DBFF020EEECFDBFF030EEECFDBFF100EEA
:102FA000DBCFE9FF110EDBCFEAFF220EE926000E90
:102FB000EA22DFCFEEFF010EDBCFEEFF020EDBCF0A
:102FC000EEFF030EDBCFEEFF040EDBCF00F0050EAD
:102FD000DBCF01F0060EDBCF02F0070EDBCF03F0F4
:102FE000D950FA0FE96EFF0EDA20EA6EEE50005C5F
:102FF000EE500158EE500258EE50035801E389D0CC
:10300000D9CFE9FFDACFEAFFEECFE6FFEECFE6FF5A
:10301000EECFE6FFEFCFE6FFB2EC00F0E552E5526F
:10302000E552E5523DC0DEFF3EC0DEFF3FC0DEFFA1
:1030300040C0DDFFDD52DD52D9CFE9FFDACFEAFF34
:10304000D880010EEE54000EEE54000EEE54000E29
:10305000EE5401E3F5D0100EDBCFE9FF110EDBCF0C
:10306000EAFF060EE926000EEA22EECF00F0EECFD0
:1030700001F0EECF02F0EFCF03F0D9CFE9FFDACFC6
:10308000EAFF0050EE5C0150EE580250EE5803503B
:10309000EE5801E3D5D0100EDBCFE9FF110EDBCFE8
:1030A000EAFF220EE926000EEA22DFCFEEFF010E34
:1030B000DBCFEEFF020EDBCFEEFF030EDBCFEEFF2A
:1030C000100EDBCFE9FF110EDBCFEAFF160EE9266B
:1030D000000EEA22040EDB50EE26050EDB50EE2237
:1030E000060EDB50EE22070EDB50EE22D950FA0F0F
:1030F000E96EFF0EDA20EA6E040EDB50EE5E050E7E
:10310000DB50EE5A060EDB50EE5A070EDB50EE5A3D
:103110005BD7100EDBCFE9FF110EDBCFEAFF160EF7
:10312000E926000EEA22FA0EDB50EE26FB0EDB50FB
:10313000EE22FC0EDB50EE22FD0EDB50EE22D9CF4C
:10314000E9FFDACFEAFFEECFE6FFEECFE6FFEECF04
:10315000E6FFEFCFE6FF66EC03F0E552E552E552FD
:10316000E552080E3DC0DBFF090E3EC0DBFF0A0E34
:103170003FC0DBFF0B0E40C0DBFF080EDBCF00F0D3
:10318000090EDBCF01F00A0EDBCF02F00B0EDBCF16
:1031900003F0005001100210031052E0100EDBCFBC
:1031A000E9FF110EDBCFEAFF160EE926000EEA2238
:1031B000EECF00F0EECF01F0EECF02F0EFCF03F054
:1031C000090ED8900332023201320032E806F9E1EA
:1031D000100EDBCFE9FF110EDBCFEAFF020EE9266E
:1031E000000EEA22EF04056A066A076AE850001634
:1031F000055001160650021607500316D950080F45
:10320000E96E000EDA20EA6EEE500026EE50012242
:10321000EE500222EE500322100EDBCFE9FF110E1A
:10322000DBCFEAFF260EE926000EEA2200C0EEFF01
:1032300001C0EEFF02C0EEFF03C0EEFF000E09D09A
:10324000100EDBCFE9FF110EDBCFEAFFEE52EF6A83
:10325000010E006E120EE15C02E2E16AE552E16EDF
:0E3260000050E552E5CFDAFFE7CFD9FF1200AC
:02326E00306AC4
:10327000316A0401FB6BFC6B020EFD6F8090120043
:10328000D9CFE6FFDACFE6FFE1CFD9FFE2CFDAFF11
:10329000E652FB0EDB5001E0EADFDF6AFD0EDB5099
:1032A0007F0BE76EFD0EE7CFDBFF315021E0FD0E17
:1032B000DBCFE6FFE66AFC0EDBCFE6FFE66AFBC487
:1032C000E6FFFCC4E6FFFE0E006E900E016E026A81
:1032D00000C0E6FFE66E02C0E6FF800EE66E000E5E
:1032E000E66E9EEC4AF0036E0B0EE15C46E243D0C4
:1032F000305021E0FD0EDBCFE6FFE66AFC0EDBCFAF
:10330000E6FFE66AFBC4E6FFFCC4E6FFEF0E006ED4
:10331000900E016E026A00C0E6FFE66E02C0E6FF94
:10332000800EE66E000EE66E9EEC4AF0036E0B0E0B
:10333000E15C23E220D0FD0EDBCFE6FFE66AFC0E67
:10334000DBCFE6FFE66AFBC4E6FFFCC4E6FFE10E66
:10335000006E900E016E026A00C0E6FFE66E02C0CB
:10336000E6FF800EE66E000EE66E9EEC4AF0036EFF
:103370000B0EE15C02E2E16AE552E16E0350800E61
:10338000E66E000EE66EEAEC48F0E552E552FC0E01
:10339000DB5001E177D0FD0EDB50040804E0FD0EA8
:1033A000DB50140804E1070EDF6E040129D1FD0E85
:1033B000DB503F0802E1316A17D0FD0EDB505F0899
:1033C00002E1306A11D0400EF36EFD0EDBCFF4FF48
:1033D000F350F45C0DE3FD0EDB50540809E3FD0EE1
:1033E000DB50400805E0306A0401FB6BFC6B47D002
:1033F000FD0EDB5040081AE1010E306E0401FB6B3C
:10340000FC6BDB0E006E900E016E026A00C0E6FFE0
:10341000E66E02C0E6FF800EE66E000EE66E9EECE3
:103420004AF0036E050EE15C20E21DD0FD0EDB507C
:10343000200828E1010E316E0401FB6BFC6BD50EF8
:10344000006E900E016E026A00C0E6FFE66E02C0DA
:10345000E6FF800EE66E000EE66E9EEC4AF0036E0E
:10346000050EE15C02E2E16AE552E16E0350800E76
:10347000E66E000EE66EEAEC48F0E552E552F36ABD
:10348000F46AF7D0620E0401FB1902E11B0EFC196D
:1034900001E1EAD00F0EFB1902E1270EFC1901E150
:1034A000E3D0580EFB1902E11B0EFC1901E1D4D048
:1034B000F70EFB1902E11A0EFC1901E1D1D0F60E4C
:1034C000FB1902E11A0EFC1901E1C2D0F50EFB193D
:1034D00002E11A0EFC1901E1B9D0A40EFB1902E1B8
:1034E0001A0EFC1901E1ADD09E0EFB1902E11A0E75
:1034F000FC1901E19FD09D0EFB1902E11A0EFC1987
:1035000001E193D09C0EFB1902E11A0EFC1901E1B6
:1035100087D09B0EFB1902E11A0EFC1901E17BD04A
:10352000920EFB1902E11A0EFC1973E0F40EFB195E
:1035300002E11A0EFC1967E0C20EFB1902E11A0E35
:10354000FC195CE0900EFB1902E11A0EFC193EE03A
:10355000FB5101E089D0FC5101E086D0FD0EDB502B
:10356000600804E1305002E0030E49D0FD0EDB504C
:10357000600804E1315002E0050E41D0FD0EDB5041
:10358000680806E1315004E0900EFB6F1A0EFC6FE4
:10359000FD0EDB50680804E1305002E0020E2FD02F
:1035A000FD0EDB506A0806E1315004E0F40EFB6FBB
:1035B0001A0EFC6FFD0EDB50700856E1305054E0DF
:1035C000040EDF6EFB6BFC6B80804ED0FD0EDB507B
:1035D000020804E1920EFB6F1A0EFC6FFD0EDB5029
:1035E000030804E0FD0EDB50FF0802E1808006D0F6
:1035F000FD0EDB50160838E1A40E2BD0020EDF6E54
:10360000FB6BFC6B31D0FD0EDB5005082DE1F50E98
:1036100020D09B0E1ED0FD0EDBCFF7F49C0E19D0F0
:10362000FD0EDBCFF8F49D0E14D0FD0EDBCFF9F4C8
:103630009E0E0FD0FD0EDBCFFAF4FB6BFC6B010E80
:1036400003D0FB6BFC6B060EDF6E0ED0F60E01D0C6
:10365000F70EFB6F1A0E07D0FB6BFC6B040EDF6ED0
:103660000F0EFB6F270EFC6FDF50016AF36E01C077
:10367000F4FFE552E552E5CFDAFFE7CFD9FF1200BC
:10368000C40E006E900E016E026A00C0E6FFE66E88
:1036900002C0E6FF800EE66E000EE66E9EEC4AF07B
:1036A000036E050EE15C02E2E16AE552E16E035051
:1036B000800EE66E000EE66EEAEC48F0E552E5524A
:1036C000020E1E101E6E0201006B82A403D0130EA8
:1036D0000211026F016B0D0E026F036B82A402D008
:1036E000600E036F040EE66EE66AFAEC43F0E552F4
:1036F000E552FD0E1E141E6E80901200D9CFE6FF1B
:10370000DACFE6FFE1CFD9FFE2CFDAFFE652E652A9
:10371000E652E652E652F8C400F0016A026A036A11
:1037200000AE03D0016802680368040ED89000362A
:10373000013602360336E806F9E102C003F001C0A3
:1037400002F000C001F0006AD8900036013602365F
:103750000336F9C404F0056A066A076A04AE02D0AB
:103760000568066806C007F005C006F004C005F04D
:10377000046A040ED8900436053606360736E80685
:10378000F9E104500026055001220650022207509C
:103790000322FAC408F0096A0A6A0B6A08AE02D06A
:1037A00009680A680AC00BF009C00AF008C009F0ED
:1037B000086A08500026095001220A5002220B50C4
:1037C000032200C0DFFF010E01C0DBFF020E02C0BA
:1037D000DBFF030E03C0DBFFF8C400F0016A026ADE
:1037E000036A00AE03D0016802680368040ED89033
:1037F0000036013602360336E806F9E1D890003685
:10380000013602360336F9C404F0056A066A076A0F
:1038100004AE03D0056806680768040ED890043625
:10382000053606360736E806F9E10450002605504D
:1038300001220650022207500322FAC408F0096A46
:103840000A6A0B6A08AE03D009680A680B68085058
:103850000026095001220A5002220B50032200C008
:10386000E6FF01C0E6FF02C0E6FF03C0E6FFFAC4C0
:103870000CF00D6A0CBE0D680CC0E6FF0DC0E6FF33
:10388000F9C40EF00F6A0EBE0F680EC0E6FF0FC03F
:10389000E6FFF8C410F0116A10BE116810C0E6FF10
:1038A00011C0E6FFF7C412F0136A12BE136812C00B
:1038B000E6FF13C0E6FFA50E146E900E156E166A95
:1038C00014C0E6FFE66E16C0E6FF800EE66E000E40
:1038D000E66E9EEC4AF0176E110EE15C02E2E16AC0
:1038E000E552E16E1750800EE66E000EE66EEAECD1
:1038F00048F0E552E552D9CFE9FFDACFEAFFEECF43
:10390000E6FFEECFE6FFEECFE6FFEFCFE6FFD9CF43
:10391000E9FFDACFEAFFEECFE6FFEECFE6FFEECF2C
:10392000E6FFEFCFE6FF8E0E006E900E016E026A8C
:1039300000C0E6FFE66E02C0E6FF800EE66E000EF7
:10394000E66E9EEC4AF0036E0D0EE15C02E2E16A67
:10395000E552E16E0350800EE66E000EE66EEAEC74
:1039600048F0E552E552D9CFE9FFDACFEAFFEECFD2
:10397000E6FFEECFE6FFEECFE6FFEFCFE6FF1DEC72
:1039800016F0E552E552E552E552E76E040EE7CF38
:10399000DBFFDB5036E0040EDBCF00F0016A00BE37
:1039A000016800C0E6FF01C0E6FFD9CFE9FFDACF2A
:1039B000EAFFEECFE6FFEECFE6FFEECFE6FFEFCF7A
:1039C000E6FF760E026E900E036E046A02C0E6FFFA
:1039D000E66E04C0E6FF800EE66E000EE66E9EEC1C
:1039E0004AF0056E0B0EE15C02E2E16AE552E16E1F
:1039F0000550800EE66E000EE66EEAEC48F0E552E9
:103A0000E5520401FD6B8090050EE15C02E2E16A83
:103A1000E552E16EE552E5CFDAFFE7CFD9FF1200BC
:103A2000D9CFE6FFDACFE6FFE1CFD9FFE2CFDAFF69
:103A3000090EE12402E3E168E652E16EF8C400F009
:103A4000016A026A036A00AE03D001680268036873
:103A5000040ED8900036013602360336E806F9E146
:103A6000D8900036013602360336F9C404F0056AF0
:103A7000066A076A04AE03D0056806680768040E84
:103A8000D8900436053606360736E806F9E10450C4
:103A90000026055001220650022207500322FAC4D4
:103AA00008F0096A0A6A0B6A08AE03D009680A6856
:103AB0000B6808500026095001220A5002220B50C0
:103AC000032200C0E6FF01C0E6FF02C0E6FF03C01C
:103AD000E6FFFAC40CF00D6A0CBE0D680CC0E6FFE0
:103AE0000DC0E6FFF9C40EF00F6A0EBE0F680EC0DF
:103AF000E6FF0FC0E6FFF8C410F0116A10BE1168AF
:103B000010C0E6FF11C0E6FF520E126E900E136E4B
:103B1000146A12C0E6FFE66E14C0E6FF800EE66E81
:103B2000000EE66E9EEC4AF0156E0F0EE15C02E2AE
:103B3000E16AE552E16E1550800EE66E000EE66E0B
:103B4000EAEC48F0E552E552020EDB6A030EDB6A4E
:103B5000040EDB6A050EDB6AD950070FE66E000E15
:103B6000DA20E66EE66A010EE66E000EE66E020EE2
:103B7000E66E35EC10F0006E060EE15C02E2E16AE2
:103B8000E552E16E0050E76E060EE7CFDBFF070E51
:103B9000DBCFE6FF080EDBCFE6FF060EDBCF00F043
:103BA000016A00BE016800C0E6FF01C0E6FF310EF9
:103BB000026E900E036E046A02C0E6FFE66E04C059
:103BC000E6FF800EE66E000EE66E9EEC4AF0056E95
:103BD000090EE15C02E2E16AE552E16E0550800EF9
:103BE000E66E000EE66EEAEC48F0E552E552FD0E98
:103BF0001E141E6E070EDBCFE6FF080EDBCFE6FFBE
:103C0000FAEC43F0E552E552070EDBCF00F0080E68
:103C1000DBCF01F0026A036AD950020FE96E000E91
:103C2000DA20EA6EEE500026EE500122EE5002221B
:103C3000EE500322020E00C0DBFF030E01C0DBFFCB
:103C4000040E02C0DBFF050E03C0DBFFD950020FDC
:103C5000E96E000EDA20EA6EEECFE6FFEECFE6FF69
:103C6000EECFE6FFEFCFE6FF1F0E006E900E016E67
:103C7000026A00C0E6FFE66E02C0E6FF800EE66E56
:103C8000000EE66E9EEC4AF0036E090EE15C02E265
:103C9000E16AE552E16E0350800EE66E000EE66EBC
:103CA000EAEC48F0E552E5520401FD6B8090090E04
:103CB000E15C02E2E16AE552E16EE552E5CFDAFF4E
:103CC000E7CFD9FF1200D9CFE6FFDACFE6FFE1CF89
:103CD000D9FFE2CFDAFF150EE12402E3E168E652F4
:103CE000E16EF8C400F0016A026A036A00AE03D014
:103CF000016802680368040ED89000360136023667
:103D00000336E806F9E1D89000360136023603366C
:103D1000F9C404F0056A066A076A04AE03D00568B0
:103D200006680768040ED89004360536063607364E
:103D3000E806F9E10450002605500122065002224F
:103D400007500322FAC408F0096A0A6A0B6A08AE2F
:103D500003D009680A680B68085000260950012240
:103D60000A5002220B50032200C0E6FF01C0E6FF0A
:103D700002C0E6FF03C0E6FFFAC40CF00D6A0CBEF9
:103D80000D680CC0E6FF0DC0E6FFF9C40EF00F6A27
:103D90000EBE0F680EC0E6FF0FC0E6FFF8C410F0BD
:103DA000116A10BE116810C0E6FF11C0E6FFFC0EDC
:103DB000126E8F0E136E146A12C0E6FFE66E14C008
:103DC000E6FF800EE66E000EE66E9EEC4AF0156E83
:103DD0000F0EE15C02E2E16AE552E16E1550800EE1
:103DE000E66E000EE66EEAEC48F0E552E552F8C4E5
:103DF00000F0016A026A036A00AE03D0016802683B
:103E00000368040ED8900036013602360336E80601
:103E1000F9E1D8900036013602360336F9C404F0D1
:103E2000056A066A076A04AE03D005680668076873
:103E3000040ED8900436053606360736E806F9E152
:103E4000045000260550012206500222075003228A
:103E5000FAC408F0096A0A6A0B6A08AE03D0096856
:103E60000A680B6808500026095001220A500222F5
:103E70000B5003220E0E00C0DBFF0F0E01C0DBFF54
:103E8000100E02C0DBFF110E03C0DBFF060EDB6A63
:103E9000070EDB6A080EDB6A090EDB6A010EDE6EB6
:103EA000DD6A0E0EDBCF00F00F0E100E110E010EAC
:103EB0000016016A026A036A005001100210031022
:103EC00001E0DFD00E0EDBCF00F00F0EDBCF01F0F4
:103ED000100EDBCF02F0110EDBCF03F0D8900332CF
:103EE000023201320032090ED89000360136023615
:103EF0000336E806F9E1012A000E022203220A0E27
:103F000000C0DBFF0B0E01C0DBFF0C0E02C0DBFFAD
:103F10000D0E03C0DBFFD9500A0FE96E000EDA2048
:103F2000EA6EEECFE6FFEECFE6FFEECFE6FFEFCF95
:103F3000E6FF1DEC16F0E552E552E552E552E76E5C
:103F4000120EE7CFDBFFD950130FE66E000EDA201A
:103F5000E66EE66A010EE66E000EE66E030EE66E93
:103F600035EC10F0006E060EE15C02E2E16AE5520B
:103F7000E16E0050E76E120EE7CFDBFFDBCF00F003
:103F8000016A00BE016800C0E6FF01C0E6FFD9502B
:103F90000A0FE96E000EDA20EA6EEECFE6FFEECFF2
:103FA000E6FFEECFE6FFEFCFE6FF010E026E036AFB
:103FB000046A056AD9500E0FE96E000EDA20EA6E27
:103FC000EE500226EE500322EE500422EE5005225F
:103FD00002C0E6FF03C0E6FF04C0E6FF05C0E6FF3F
:103FE000DD0E066E8F0E076E086A06C0E6FFE66EEF
:103FF00008C0E6FF800EE66E000EE66E9EEC4AF00C
:10400000096E0F0EE15C02E2E16AE552E16E0950D1
:10401000800EE66E000EE66EEAEC48F0E552E552E0
:104020000A0EDBCF00F00B0EDBCF01F00C0EDBCF66
:1040300002F00D0EDBCF03F00106000E025A035A08
:104040000A0E00C0DBFF0B0E01C0DBFF0C0E02C02E
:10405000DBFF0D0E03C0DBFFD9500A0FE96E000E27
:10406000DA20EA6EEECFE6FFEECFE6FFEECFE6FF18
:10407000EFCFE6FF1DEC16F0E552E552E552E552B2
:10408000D8D00E0EDBCF3DF00F0EDBCF3EF0100E82
:10409000DBCF3FF0110EDBCF40F0D89040323F3203
:1040A0003E323D32426A020E436E446A456A85ECF6
:1040B0004BF00A0E39C0DBFF0B0E3AC0DBFF0C0ED3
:1040C0003BC0DBFF0D0E3CC0DBFFD9500A0FE96E91
:1040D000000EDA20EA6EEECFE6FFEECFE6FFEECF7F
:1040E000E6FFEFCFE6FF1DEC16F0E552E552E55294
:1040F000E552E76E120EE7CFDBFFD950130FE66EE5
:10410000000EDA20E66EE66A010EE66E000EE66E3E
:10411000030EE66E35EC10F0006E060EE15C02E276
:10412000E16AE552E16E0050E76E120EE7CFDBFF69
:10413000DBCF00F0016A00BE016800C0E6FF01C0ED
:10414000E6FFD9500A0FE96E000EDA20EA6EEECFD4
:10415000E6FFEECFE6FFEECFE6FFEFCFE6FF0E0E77
:10416000DBCF02F00F0EDBCF03F0100EDBCF04F03D
:10417000110EDBCF05F00206000E035A045A055A51
:1041800002C0E6FF03C0E6FF04C0E6FF05C0E6FF8D
:10419000BD0E066E8F0E076E086A06C0E6FFE66E5D
:1041A00008C0E6FF800EE66E000EE66E9EEC4AF05A
:1041B000096E0F0EE15C02E2E16AE552E16E095020
:1041C000800EE66E000EE66EEAEC48F0E552E5522F
:1041D000D9500A0FE96E000EDA20EA6EEECFE6FF44
:1041E000EECFE6FFEECFE6FFEFCFE6FF1DEC16F0D9
:1041F000E552E552E552E552E76E120EE7CFDBFFDE
:1042000082B41BD0D950130FE66E000EDA20E66E92
:10421000E66A010EE66E000EE66E030EE66EFDEC3B
:1042200012F0006E060EE15C02E2E16AE552E16E18
:104230000050E76E120EE7CFDBFFD9CFE9FFDACFF0
:10424000EAFFEE50ED1001E131D20001AD6BAE6B33
:10425000CFEC44F0120EF3CFDBFF040EDB6A050E49
:10426000DB6A040EDBCF00F0050EDBCF01F0D89047
:10427000015004E6500E005C000E015801E36BD1C2
:10428000040EDBCF02F0050EDBCF03F0040ED89056
:1042900002360336E806FBE100010250AD5D035033
:1042A000AE5901E258D1BA0E006E8F0E016E026A4D
:1042B00000C0E6FFE66E02C0E6FF800EE66E000E6E
:1042C000E66E9EEC4AF0036E050EE15C02E2E16AE6
:1042D000E552E16E0350800EE66E000EE66EEAECEB
:1042E00048F0E552E552020EDB6A030EDB6A020E6D
:1042F000DBCF00F0030EDBCF01F0D890015004E6D5
:10430000100E005C000E01585BE2040EDBCF04F0DF
:10431000050EDBCF05F0040ED89004360536E8060E
:10432000FBE1020EDB500424026E030EDB5005207D
:10433000036E00010250AD5D0350AE5941E3040E1F
:10434000DBCF00F0050EDBCF01F0040ED890003675
:104350000136E806FBE1020EDB500024E96E030E95
:10436000DB500120EA6E000EE926010EEA22EF5032
:10437000E66EE66AB40E026E8F0E036E046A02C029
:10438000E6FFE66E04C0E6FF800EE66E000EE66E07
:104390009EEC4AF0056E070EE15C02E2E16AE5522E
:1043A000E16E0550800EE66E000EE66EEAEC48F017
:1043B000E552E552020EDB2A030E99E3DB2A97D77A
:1043C000B00E006E8F0E016E026A00C0E6FFE66E50
:1043D00002C0E6FF800EE66E000EE66E9EEC4AF02E
:1043E000036E050EE15C02E2E16AE552E16E035004
:1043F000800EE66E000EE66EEAEC48F0E552E552FD
:10440000020EDB6A030EDB6A020EDBCF00F0030E46
:10441000DBCF01F0D890015004E6100E005C000ED6
:10442000015801E391D0040EDBCF04F0050EDBCF81
:1044300005F0040ED89004360536E806FBE1020EBE
:10444000DB500424026E030EDB500520036E0001D6
:104450000250AD5D0350AE5901E276D0040EDBCFC1
:1044600000F0050EDBCF01F0040ED89000360136C7
:10447000E806FBE1020EDB500024E96E030EDB5080
:104480000120EA6E000EE926010EEA22EF50200814
:1044900034E2040EDBCF00F0050EDBCF01F0040E9A
:1044A000D89000360136E806FBE1020EDB5000240E
:1044B000E96E030EDB500120EA6E000EE926010EC4
:1044C000EA22EF50E66EE66AAD0E026E8F0E036EC4
:1044D000046A02C0E6FFE66E04C0E6FF800EE66EE8
:1044E000000EE66E9EEC4AF0056E070EE15C02E2FD
:1044F000E16AE552E16E055018D0AB0E006E8F0EEA
:10450000016E026A00C0E6FFE66E02C0E6FF800EA2
:10451000E66E000EE66E9EEC4AF0036E050EE15C60
:1045200002E2E16AE552E16E0350800EE66E000E93
:10453000E66EEAEC48F0E552E552020EDB2A030E85
:1045400001E262D7DB2A60D7040EDB2A050E01E206
:1045500088D6DB2A86D6A90E006E8F0E016E026AFF
:1045600000C0E6FFE66E02C0E6FF800EE66E000EBB
:10457000E66E9EEC4AF0036E050EE15C02E2E16A33
:10458000E552E16E0350800EE66E000EE66EEAEC38
:1045900048F0E552E552ADC000F0AEC001F0026A4D
:1045A000036AD950060FE96E000EDA20EA6EEE506B
:1045B0000026EE500122EE500222EE500322060E9B
:1045C00000C0DBFF070E01C0DBFF080E02C0DBFFEF
:1045D000090E03C0DBFFD950060FE96E000EDA208A
:1045E000EA6E000EEE5C010EEE58000EEE58000E64
:1045F000EE5802E3DE6ADD6A120EDBCF00F0016ADC
:1046000000BE0168FE0E001804E1015002E1DE6AFE
:10461000DD6A82B41CD0D950130FE66E000EDA208A
:10462000E66EADC0E6FFAEC0E6FF000EE66E010E20
:10463000E66EFDEC12F0006E060EE15C02E2E16A4D
:10464000E552E16E0050E76E120EE7CFDBFF120E6F
:10465000DB5001E1F2D5120EDBCF00F0016A00BEA3
:10466000016800C0E6FF01C0E6FF990E026E8F0EE2
:10467000036E046A02C0E6FFE66E04C0E6FF800E29
:10468000E66E000EE66E9EEC4AF0056E070EE15CEB
:1046900002E2E16AE552E16E0550800EE66E000E20
:1046A000E66EEAEC48F0E552E552C7D50E0EDBCFD8
:1046B00000F00F0E100E110E010E0016016A026AB4
:1046C000036A00500110021003101DE182B436D0BD
:1046D000D950130FE66E000EDA20E66EE66A010E80
:1046E000E66E000EE66E030EE66EFDEC12F0006E56
:1046F000060EE15C02E2E16AE552E16E0050E76E0F
:10470000120EE7CFDBFF82B419D0D950130FE66E3B
:10471000000EDA20E66E000EE66EE66AE66EE66AE7
:10472000FDEC12F0006E060EE15C02E2E16AE55279
:10473000E16E0050E76E120EE7CFDBFF120EDB508A
:104740002AE0120EDBCF00F0016A00BE016800C053
:10475000E6FF01C0E6FF840E026E8F0E036E046A50
:1047600002C0E6FFE66E04C0E6FF800EE66E000EB5
:10477000E66E9EEC4AF0056E070EE15C02E2E16A2D
:10478000E552E16E0550800EE66E000EE66EEAEC34
:1047900048F0E552E552D950060FE96E000EDA20D6
:1047A000EA6EEECFE6FFEECFE6FFEECFE6FFEFCF0D
:1047B000E6FF6A0E006E8F0E016E026A00C0E6FF11
:1047C000E66E02C0E6FF800EE66E000EE66E9EEC20
:1047D0004AF0036E090EE15C02E2E16AE552E16E25
:1047E0000350800EE66E000EE66EEAEC48F0E552ED
:1047F000E552B4D80401FD6B8090150EE15C02E235
:10480000E16AE552E16EE552E5CFDAFFE7CFD9FF85
:104810001200610E006E8F0E016E026A00C0E6FF8C
:10482000E66E02C0E6FF800EE66E000EE66E9EECBF
:104830004AF0036E050EE15C02E2E16AE552E16EC8
:104840000350800EE66E000EE66EEAEC48F0E5528C
:10485000E552E66A010EE66EE66A000EE66E020EAC
:10486000E66E5BEC49F0006E050EE15C02E2E16A87
:10487000E552E16E0050FDC400F2010EE66EE66AFC
:10488000FAEC43F0E552E5520401FD6B1200550EBF
:10489000006E8F0E016E026A00C0E6FFE66E02C077
:1048A000E6FF800EE66E000EE66E9EEC4AF0036EAA
:1048B000050EE15C02E2E16AE552E16E0350800E12
:1048C000E66E000EE66EEAEC48F0E552E552E66A66
:1048D000010EE66EE66A000EE66E020EE66E5BEC18
:1048E00049F0006E050EE15C02E2E16AE552E16E1C
:1048F0000050FDC400F2010EE66EE66AFAEC43F0E9
:10490000E552E55280900401FD6B12004A0E006EE4
:104910008F0E016E026A00C0E6FFE66E02C0E6FF7F
:10492000800EE66E000EE66E9EEC4AF0036E050EFB
:10493000E15C02E2E16AE552E16E0350800EE66E50
:10494000000EE66EEAEC48F0E552E5520401FA6B1F
:10495000F96BF86B80900401FD6B1200D9CFE6FF74
:10496000DACFE6FFE1CFD9FFE2CFDAFFE652E65237
:10497000E652E652E6520401FA2B0F0EE76EFA19E0
:10498000E8AE02D0FA3503D0E750D880FA550FE2EE
:10499000FA6BF92B010EE76EF919E8AE02D0F93582
:1049A00003D0E750D880F95502E2F96BF82BF8C430
:1049B00000F0016A026A036A00AE03D0016802686F
:1049C0000368040ED8900036013602360336E80636
:1049D000F9E102C003F001C002F000C001F0006A7A
:1049E000D8900036013602360336F9C404F0056A61
:1049F000066A076A04AE02D00568066806C007F0BA
:104A000005C006F004C005F0046A040ED890043610
:104A1000053606360736E806F9E10450002605504B
:104A200001220650022207500322FAC408F0096A44
:104A30000A6A0B6A08AE02D009680A680AC00BF05D
:104A400009C00AF008C009F0086A08500026095099
:104A500001220A5002220B50032200C0DFFF010E88
:104A600001C0DBFF020E02C0DBFF030E03C0DBFF51
:104A7000FAC400F0016A00BE016800C0E6FF01C090
:104A8000E6FFF9C402F0036A02BE036802C0E6FF53
:104A900003C0E6FFF8C404F0056A04BE056804C05C
:104AA000E6FF05C0E6FFF7C406F0076A06BE076822
:104AB00006C0E6FF07C0E6FF2B0E086E8F0E096EDC
:104AC0000A6A08C0E6FFE66E0AC0E6FF800EE66EE0
:104AD000000EE66E9EEC4AF00B6E0D0EE15C02E2FB
:104AE000E16AE552E16E0B50800EE66E000EE66E56
:104AF000EAEC48F0E552E552D9CFE9FFDACFEAFF18
:104B0000EECFE6FFEECFE6FFEECFE6FFEFCFE6FF1C
:104B1000D9CFE9FFDACFEAFFEECFE6FFEECFE6FF2F
:104B2000EECFE6FFEFCFE6FF8E0E006E900E016E29
:104B3000026A00C0E6FFE66E02C0E6FF800EE66E87
:104B4000000EE66E9EEC4AF0036E0D0EE15C02E292
:104B5000E16AE552E16E0350800EE66E000EE66EED
:104B6000EAEC48F0E552E552D9CFE9FFDACFEAFFA7
:104B7000EECFE6FFEECFE6FFEECFE6FFEFCFE6FFAC
:104B80001DEC16F0E552E552E552E552E76E040ED3
:104B9000E7CFDBFFDB5036E0040EDBCF00F0016A2D
:104BA00000BE016800C0E6FF01C0E6FFD9CFE9FF03
:104BB000DACFEAFFEECFE6FFEECFE6FFEECFE6FF7D
:104BC000EFCFE6FF760E026E900E036E046A02C00F
:104BD000E6FFE66E04C0E6FF800EE66E000EE66EAF
:104BE0009EEC4AF0056E0B0EE15C02E2E16AE552D2
:104BF000E16E0550800EE66E000EE66EEAEC48F0BF
:104C0000E552E5520401FD6B050EE15C02E2E16A4A
:104C1000E552E16EE552E5CFDAFFE7CFD9FF1200AA
:104C20000F01006B016B086B096B0A6B0B6BA4C463
:104C300000F0016A026A036A000E006C011E012284
:104C4000021E0222031E0322A5C404F0056A066A9E
:104C5000076A180ED8900436053606360736E80679
:104C6000F9E10450002605500122065002220750A7
:104C70000322A6C408F0096A0A6A0B6A100ED890CB
:104C8000083609360A360B36E806F9E108500026E0
:104C9000095001220A5002220B500322A7C43DF002
:104CA0003E6A3F6A406A426A010E436E446A456A40
:104CB00085EC4BF0005039240F010C6F01503A2065
:104CC0000D6F02503B200E6F03503C200F6F0CCF36
:104CD000E6FF0DCFE6FF0ECFE6FFE66E0CCFE6FF58
:104CE0000DCFE6FF0ECFE6FFE66E150E006E910EBD
:104CF000016E026A00C0E6FFE66E02C0E6FF800EAB
:104D0000E66E000EE66E9EEC4AF0036E0D0EE15C60
:104D100002E2E16AE552E16E0350800EE66E000E9B
:104D2000E66EEAEC48F0E552E552306A316A326AE2
:104D3000336A346A356A020E366E0F01146B809046
:104D40001200D9CFE6FFDACFE6FFE1CFD9FFE2CFFD
:104D5000DAFFE652FB0EDB5001E062DFDF6AFC0E99
:104D6000DB5007E0FD0EDB507F0BE76EFD0EE7CF5B
:104D7000DBFFFC0EDB506BE0FD0EDB50040804E0B3
:104D8000FD0EDB50140803E1070EDF6EABD0FD0E05
:104D9000DB503F0802E1316A23D0FD0EDB505F0893
:104DA00010E0400EF36EFD0EDBCFF4FFF350F45C29
:104DB0000AE3FD0EDB505E0806E3FD0EDB50400803
:104DC00002E0306A0DD0FD0EDB50400803E1010E19
:104DD000306E06D0FD0EDB50200804E1010E316E6E
:104DE000336A32D0FD0EDB50650806E1315004E035
:104DF000346A356A010E27D0FD0EDB506E0802E1E1
:104E0000020E336EFD0EDB50700806E1305004E0F8
:104E1000346A356A030E336EFD0EDB50700807E10D
:104E2000315005E08080346A356A040E0CD0FD0EE6
:104E3000DB5072080CE131500AE080802A0E346E9B
:104E40001C0E356E050E336EF36AF46A53D0335080
:104E5000050A41E0010A3CE0070A15E0010A0AE000
:104E6000030A02E0010A41D0FD0EDBCFE6FF49D87C
:104E7000E5522CD08080FD0EDBCFE6FFC0D9E55295
:104E8000DF6E336A32D08080E66A010EE66EE66A33
:104E9000000EE66E020EE66E5BEC49F0006E050E4B
:104EA000E15C02E2E16AE552E16E0050020E1E1082
:104EB0001E6E36C000F2010EE66EE66AFAEC43F0B2
:104EC000E552E552FD0E1E141E6E080EDF6E0DD06B
:104ED0008090DF6A0AD0FD0EDB50080806E1809062
:104EE000DF6A366A336A346A356ADF50016AF36E04
:104EF00001C0F4FFE552E552E5CFDAFFE7CFD9FF75
:104F00001200D9CFE6FFDACFE6FFE1CFD9FFE2CF3B
:104F1000DAFFE652DF6A2A0E341802E11C0E351859
:104F200001E165D10F0E341802E1270E351801E1B9
:104F30005ED1760E341802E10E0E351801E153D120
:104F4000750E341802E10E0E351801E147D1AC0E92
:104F5000341802E10D0E351801E149D1480E34181C
:104F600002E10D0E351801E136D10C0E341802E1C4
:104F7000070E351801E129D10B0E341802E1070E96
:104F8000351801E11BD10A0E341802E1070E35185D
:104F900001E10FD1090E341802E1070E351801E1C5
:104FA00003D1EE0E341802E1030E351801E1A8D04A
:104FB000ED0E341802E1030E351801E19AD0EC0E23
:104FC000341802E1030E351801E18ED0EB0E3418CF
:104FD00002E1030E351801E182D0EA0E341802E135
:104FE000030E351801E176D0E90E341802E1030E04
:104FF00035186BE0345001E0FAD0355001E0F7D0BD
:10500000FD0EDB5005E1315003E0DF6A0A0E08D0E7
:10501000FD0EDB50020806E1315004E0DF6A140E99
:10502000346ED7D0200EF36EFD0EDBCFF4FFF350BD
:10503000F45C0DE3FD0EDB502F0809E3315007E06F
:10504000FD0EDB50E00F0F01006FDF6AC1D0400E94
:10505000F36EFD0EDBCFF4FFF350F45C0DE3FD0EB9
:10506000DB504F0809E3315007E0FD0EDB50C00F65
:105070000F01016FDF6AAFD0FD0EDB50350807E18D
:10508000315005E0DF6AAC0E346E0D0E0AD0FD0E15
:10509000DB500D0808E1315006E0DF6ABC0E346ECB
:1050A000020E356EA3D0FD0EDB50100804E1315026
:1050B00002E0E90E22D0FD0EDB50180801E097D087
:1050C000315001E194D0090E7DD0FD0EDBCF02FFFF
:1050D000EA0E13D0FD0EDBCF03FFEB0E0ED0FD0E5C
:1050E000DBCF04FFEC0E09D0FD0EDBCF05FFED0E8C
:1050F00004D0FD0EDBCF06FFEE0E346E030E71D032
:10510000FD0EDBCF07FF04CF00F0016A026A036ADD
:10511000000E006C011E0122021E0222031E032249
:1051200005CF04F0056A066A076A180ED89004369F
:10513000053606360736E806F9E104500026055024
:105140000122065002220750032206CF08F0096A06
:105150000A6A0B6A100ED890083609360A360B36E2
:10516000E806F9E108500026095001220A500222FF
:105170000B50032207CF3DF03E6A3F6A406A426A05
:10518000010E436E446A456A85EC4BF000503924A9
:105190000F01086F01503A20096F02503B200A6F3F
:1051A00003503C200B6F17D0FD0EDBCF13FF0A0E10
:1051B00009D0FD0EDBCF12FF0B0E04D0FD0EDBCFAE
:1051C00011FF0C0E346E070E0CD0FD0EDBCF10FF5E
:1051D000346A356A0BD0346A356A09D0760E346E7B
:1051E0000E0E356E04D0346A356ADF6A8090DF5067
:1051F000E552E552E5CFDAFFE7CFD9FF1200D9CF6C
:10520000E6FFDACFE6FFE1CFD9FFE2CFDAFFE652E1
:105210000F0E341802E1270E351823E0BC0E3418A7
:1052200002E1020E351819E0AC0E341802E10D0E41
:10523000351811E0140E341801E1355007E00A0E5C
:1052400034180EE135500CE1030E08D0050EDF6E68
:10525000346A356A06D0010E01D0020EDF6E01D02D
:10526000DF6ADF50E552E552E5CFDAFFE7CFD9FF3D
:105270001200FD0E1E141E6E050EE66EE66A840E0A
:10528000E66E040EE66E000EE66E020EE66E30EC82
:1052900049F0006E060EE15C02E2E16AE552E16E61
:1052A0000050050EE66EE66AFAEC43F0E552E55270
:1052B000130EE66EE66A890EE66E040EE66E000ECA
:1052C000E66E020EE66E30EC49F0006E060EE15C12
:1052D00002E2E16AE552E16E0050130EE66EE66A04
:1052E000FAEC43F0E552E552020E1E101E6E0D0E52
:1052F000E66EE66A9C0EE66E040EE66E000EE66E44
:10530000020EE66E30EC49F0006E060EE15C02E241
:10531000E16AE552E16E00500D0EE66EE66AFAECC7
:1053200043F0E552E552FD0E1E141E6E80901200F1
:10533000020E1E101E6EE66A010EE66EE66A000E92
:10534000E66E020EE66E5BEC49F0006E050EE15C67
:1053500002E2E16AE552E16E00500201110E006FB7
:1053600001690F0114A503D00201010E046F0F01A2
:1053700014A103D00201020E066F0F0114A303D083
:105380000201020E066F82A403D00201080E066F0E
:1053900014CF36F002CF0BF203CF0CF204CF0DF294
:1053A00005CF0EF206CF0FF207CF10F2140EE66E05
:1053B000E66AFAEC43F0E552E552FD0E1E141E6E4D
:1053C00080901200D9CFE6FFDACFE6FFE1CFD9FF18
:1053D000E2CFDAFFE652E652E652E652E65208CF54
:1053E000DFFF010E09CFDBFF020E0ACFDBFF030E4A
:1053F0000BCFDBFF080EE96E0F0EEA6EEE500F01C9
:105400000C5DEE500D59EE500E59EE500F5905E25D
:10541000010E366E040E1411146F100EE96E0F0E8D
:10542000EA6E0851EE24006E0951EE20016E0A5119
:10543000EE20026E0B51EE20036E00500C5D015009
:105440000D5902500E5903500F5905E2010E366EE8
:10545000040E1411146F366AD9CFE9FFDACFEAFFD0
:10546000EECFE6FFEECFE6FFEECFE6FFEFCFE6FFB3
:105470001DEC16F0E552E552E552E552E76E040EDA
:10548000E7CFDBFFDB5006E0010E366E040E0F01A6
:105490001411146F3650016A36C0F3FF01C0F4FFD7
:1054A000050EE15C02E2E16AE552E16EE552E5CF0C
:1054B000DAFFE7CFD9FF1200D9CFE6FFDACFE6FF58
:1054C000E1CFD9FFE2CFDAFF0F0EE12402E3E1687A
:1054D000E652E16E808076DF020EF3CFDBFF030E33
:1054E000F4CFDBFFD950020FE96E000EDA20EA6E2E
:1054F000EE50ED1001E0E9D010CF3DF011CF3EF0BD
:1055000012CF3FF013CF40F0426A010E436E446A5F
:10551000456AEAEC4BF00B0E3DC0DBFF0C0E3EC0C3
:10552000DBFF10CF3DF011CF3EF012CF3FF013CF95
:1055300040F0426A010E436E446A456AEAEC4BF061
:105540000D0E39C0DBFF0E0E3AC0DBFFFD0E1E1440
:105550001E6E040EDB6A050EDB6A060EDB6A070EA2
:10556000DB6ADE6ADD6ADECF00F0DDCF01F00B0E14
:10557000DBCF02F00C0EDBCF03F001500318E8AED6
:1055800002D0033404D00250005C0350015870E292
:105590000B0EDBCF00F00C0EDBCF01F00006000E8F
:1055A000015A0050DF1810E10150DE52DD180CE105
:1055B000D9500D0FE96E000EDA20EA6EEE50ED10B4
:1055C00003E1020E1E101E6ED950090FE66E000E8A
:1055D000DA20E66EE66A010EE66E000EE66E020E58
:1055E000E66E35EC10F0006E060EE15C02E2E16A58
:1055F000E552E16E0050E76E080EE7CFDBFFDB50AF
:1056000064E1090EDBCFE6FF0A0EDBCFE6FFFAEC22
:1056100043F0E552E552090EDBCF00F00A0EDBCF76
:1056200001F0026A036AD950040FE96E000EDA2015
:10563000EA6EEE500026EE500122EE500222EE50AD
:105640000322040E00C0DBFF050E01C0DBFF060EC7
:1056500002C0DBFF070E03C0DBFF0F01092B000EAA
:105660000A230B23DF2A010E01E27DD7DB2A7BD739
:105670000D0EDBCF00F00E0EDBCF01F0013466E241
:1056800000500008000E015461E2D950090FE66E87
:10569000000EDA20E66E0D0EDBCFE6FF0E0EDBCF3E
:1056A000E6FF000EE66E020EE66E35EC10F0006EC0
:1056B000060EE15C02E2E16AE552E16E0050E76E3F
:1056C000080EE7CFDBFFDB500DE0040E0F011411D5
:1056D000146F71EC2FF0020EDBCF00F0030EDBCF66
:1056E00001F03CD0020E1E101E6E0D0EDBCFE6FF49
:1056F0000E0EDBCFE6FFFAEC43F0E552E552090E61
:10570000DBCF00F00A0EDBCF01F0026A036AD9504A
:10571000040FE96E000EDA20EA6EEE500026EE501D
:105720000122EE500222EE500322040E00C0DBFFE5
:10573000050E01C0DBFF060E02C0DBFF070E03C033
:10574000DBFF0F01092B000E0A230B23FD0E1E1495
:105750001E6E366A80903650006E016A00C0F3FFFC
:1057600001C0F4FF0F0EE15C02E2E16AE552E16E76
:10577000E552E5CFDAFFE7CFD9FF1200D9CFE6FF38
:10578000DACFE6FFE1CFD9FFE2CFDAFF0F0EE12457
:1057900002E3E168E652E16E366A14DE0B0EF3CFE7
:1057A000DBFF0C0EF4CFDBFFD9500B0FE96E000EC0
:1057B000DA20EA6EEE50ED1007E00B0EDBCF00F0C2
:1057C0000C0EDBCF01F0A4D0060EDB6A070EDB6AFD
:1057D000080EDB6A090EDB6A010EDE6EDD6AD9CFC8
:1057E000E9FFDACFEAFFEE50ED1001E196D00001BB
:1057F000AD6BAE6BCFEC44F00B0EF3CFDBFF0C0EBA
:10580000F4CFDBFFADC000F0AEC001F0026A036A66
:10581000D950060FE96E000EDA20EA6EEE5000262F
:10582000EE500122EE500222EE500322060E00C07E
:10583000DBFF070E01C0DBFF080E02C0DBFF090E15
:1058400003C0DBFFD950060FE96E000EDA20EA6EC6
:105850000F011051EE5C1151EE581251EE581351D8
:10586000EE5802E3DE6ADD6AD9500B0FE96E000ED6
:10587000DA20EA6EFE0EEE1804E1ED5002E1DE6A77
:10588000DD6A81BC02D0DE6ADD6A0001000EAD5D1A
:10589000010EAE592DE2ADC000F0AEC001F0000E19
:1058A000D8800056010E015600C0E6FF01C0E6FF99
:1058B000ADC0E9FFAEC0EAFFE906000EEA5A000EED
:1058C000E926010EEA22EF50E66E000EAD25026ECB
:1058D000010EAE21036E02C0E6FFE66E5BEC49F0FE
:1058E000046E050EE15C02E2E16AE552E16E0450ED
:1058F00096D80A0EF3CFDBFFDB5001E170D7010E23
:10590000366E040E0F011411146F3650006E016ACA
:1059100000C0F3FF01C0F4FF07D082A402D0010E43
:10592000366E8090F36AF46A0F0EE15C02E2E16A7F
:10593000E552E16EE552E5CFDAFFE7CFD9FF12007D
:10594000E66A010EE66EE66A000EE66E020EE66E8E
:105950005BEC49F0006E050EE15C02E2E16AE552A3
:10596000E16E005036C000F2010EE66EE66AFAEC17
:1059700043F0E552E552366A12000F01086B096BDD
:105980000A6B0B6B146B106B116B126B136B8090AB
:10599000366A1200D9CFE6FFDACFE6FFE1CFD9FFB2
:1059A000E2CFDAFFE652E652E652E652E6520F0145
:1059B000092B000E0A230B2308CFDFFF010E09CFAE
:1059C000DBFF020E0ACFDBFF030E0BCFDBFFD9CFCD
:1059D000E9FFDACFEAFFEECFE6FFEECFE6FFEECF4C
:1059E000E6FFEFCFE6FF1DEC16F0E552E552E5527B
:1059F000E552E76E040EE7CFDBFFDB5003E0010E5C
:105A0000366E01D0366A050EE15C02E2E16AE552CB
:105A1000E16EE552E5CFDAFFE7CFD9FF1200D9CF2B
:105A2000E6FFDACFE6FFE1CFD9FFE2CFDAFF130ED0
:105A3000E12402E3E168E652E16E08CF3DF009CFD0
:105A40003EF00ACF3FF00BCF40F0426A010E436EAA
:105A5000446A456AEAEC4BF00A0E3DC0DBFF0B0ED0
:105A60003EC0DBFF0C0E3FC0DBFF0D0E40C0DBFF76
:105A7000110EDB6A120EDB6AA5DC040EF3CFDBFF2E
:105A8000050EF4CFDBFFD950040FE96E000EDA20CB
:105A9000EA6EEE50ED1005E0040EDBCF00F0050ECF
:105AA0000ED20A0EDBCF00F00B0E0C0E0D0E010E07
:105AB0000016016A026A036A005001100210031006
:105AC00001E0ACD00A0EDBCF00F00B0EDBCF01F013
:105AD0000C0EDBCF02F00D0EDBCF03F0D8900332BB
:105AE000023201320032090ED890003601360236F9
:105AF0000336E806F9E1012A000E02220322060E0F
:105B000000C0DBFF070E01C0DBFF080E02C0DBFF99
:105B1000090E03C0DBFFD950060FE96E000EDA2034
:105B2000EA6EEECFE6FFEECFE6FFEECFE6FFEFCF79
:105B3000E6FF1DEC16F0E552E552E552E552E76E40
:105B4000100EE7CFDBFFDB5007E0100EDBCF00F0DD
:105B5000016A00AEB6D1A3D1D9500E0FE66E000E89
:105B6000DA20E66EE66A010EE66E000EE66E030EC1
:105B7000E66E35EC10F0006E060EE15C02E2E16AC2
:105B8000E552E16E0050E76E100EE7CFDBFFDB5011
:105B900007E0100EDBCF00F0016A00AE92D17FD19A
:105BA000060EDBCF00F0070EDBCF01F0080EDBCFD7
:105BB00002F0090EDBCF03F00106000E025A035A71
:105BC000060E00C0DBFF070E01C0DBFF080E02C09F
:105BD000DBFF090E03C0DBFFD950060FE96E000E94
:105BE000DA20EA6EEECFE6FFEECFE6FFEECFE6FF7D
:105BF000EFCFE6FF1DEC16F0E552E552E552E55217
:105C0000E76E100EE7CFDBFFDB5001E1B8D0100EDE
:105C1000DBCF00F0016A00AE54D141D10A0EDBCFD8
:105C20003DF00B0EDBCF3EF00C0EDBCF3FF00D0E48
:105C3000DBCF40F0D89040323F323E323D32426AB4
:105C4000020E436E446A456A85EC4BF0060E39C07D
:105C5000DBFF070E3AC0DBFF080E3BC0DBFF090E7F
:105C60003CC0DBFFD950060FE96E000EDA20EA6E69
:105C7000EECFE6FFEECFE6FFEECFE6FFEFCFE6FF9B
:105C80001DEC16F0E552E552E552E552E76E100EB6
:105C9000E7CFDBFFDB5007E0100EDBCF00F0016A3F
:105CA00000AE0FD1FCD0D9500E0FE66E000EDA20F8
:105CB000E66EE66A010EE66E000EE66E030EE66E16
:105CC00035EC10F0006E060EE15C02E2E16AE5528E
:105CD000E16E0050E76E100EE7CFDBFFDB5007E010
:105CE000100EDBCF00F0016A00AEEBD0D8D0D95057
:105CF000060FE96E000EDA20EA6EEECFE6FFEECF79
:105D0000E6FFEECFE6FFEFCFE6FF1DEC16F0E55223
:105D1000E552E552E552E76E100EE7CFDBFFDB50B0
:105D200007E0100EDBCF00F0016A00AECAD0B7D09A
:105D300082B41BD0D9500E0FE66E000EDA20E66E4C
:105D4000E66A010EE66E000EE66E030EE66EFDECF0
:105D500012F0006E060EE15C02E2E16AE552E16ECD
:105D60000050E76E100EE7CFDBFF100EDB5007E0B0
:105D7000100EDBCF00F0016A00AEA3D090D082B449
:105D80001BD0D9500E0FE66E000EDA20E66EE66AE2
:105D9000010EE66E000EE66E010EE66EFDEC12F0F0
:105DA000006E060EE15C02E2E16AE552E16E00502F
:105DB000E76E100EE7CFDBFF100EDB500EE0010E9A
:105DC000F36E110EF3CFDBFF120EDB6A100EDBCF8A
:105DD00000F0016A00AE75D062D00A0EDBCF00F091
:105DE0000B0E0C0E0D0E010E0016016A026A036AFC
:105DF000005001100210031027E182B41BD0D950CB
:105E00000E0FE66E000EDA20E66EE66A010EE66E12
:105E1000000EE66E030EE66EFDEC12F0006E060E4E
:105E2000E15C02E2E16AE552E16E0050E76E100EBD
:105E3000E7CFDBFF100EDB5007E0100EDBCF00F0EA
:105E4000016A00AE3ED02BD082B419D0D9500E0FCB
:105E5000E66E000EDA20E66E000EE66EE66AE66E8C
:105E6000E66AFDEC12F0006E060EE15C02E2E16A09
:105E7000E552E16E0050E76E100EE7CFDBFF100E2B
:105E8000DB500FE0010EF36E110EF3CFDBFF120EAD
:105E9000DB6A100EDBCF00F0016A00AE12D00168A1
:105EA00010D0D950110FE96E000EDA20EA6EEE50D4
:105EB000ED1001E16FDD110EDBCF00F0120EDBCF34
:105EC00001F000C0F3FF01C0F4FF130EE15C02E239
:105ED000E16AE552E16EE552E5CFDAFFE7CFD9FF9F
:105EE0001200E66A010EE66EE66A000EE66E020E2B
:105EF000E66E5BEC49F0006E050EE15C02E2E16AE1
:105F0000E552E16E00500201010E006F020E1E10FC
:105F10001E6E010EE66EE66AFAEC43F0E552E552BB
:105F2000FD0E1E141E6E1200D9CFE6FFDACFE6FF7B
:105F3000E1CFD9FFE2CFDAFFE652E652E6520F0197
:105F4000020E116F076F04CF00F0016A026A036A44
:105F5000000E006C011E0122021E0222031E0322FB
:105F600005CF04F0056A066A076A180ED890043651
:105F7000053606360736E806F9E1045000260550D6
:105F80000122065002220750032206CF08F0096AB8
:105F90000A6A0B6A100ED890083609360A360B3694
:105FA000E806F9E108500026095001220A500222B1
:105FB0000B50032207CF3DF03E6A3F6A406A426AB7
:105FC000010E436E446A456A85EC4BF0005039245B
:105FD0000F01086F01503A20096F02503B200A6FF1
:105FE00003503C200B6FDE6ADD6ADECF00F0DDCFB0
:105FF00001F0140E005C000E015851E2E66ADECF9B
:10600000E9FFDDCFEAFF010EE926000EEA22AD0E20
:10601000E926040EEA22EF50E66EDECFE9FFDDCF7F
:10602000EAFFAD0EE926040EEA22EF50E66EA1EC7F
:1060300026F0E552E552E552020EF3CFDBFFDBCF4F
:10604000E6FFE66A0D0E006E910E016E026A00C058
:10605000E6FFE66E02C0E6FF800EE66E000EE66E1C
:106060009EEC4AF0036E070EE15C02E2E16AE55243
:10607000E16E0350800EE66E000EE66EEAEC48F02C
:10608000E552E552DECF00F0DDCF01F0020E002632
:10609000000E012200C0DEFF01C0DDFFA6D7E552E1
:1060A000E552E552E552E5CFDAFFE7CFD9FF12001E
:1060B000D9CFE6FFDACFE6FFE1CFD9FFE2CFDAFFB3
:1060C0000A0EE12402E3E168E652E16EDF6A010EA6
:1060D000DB6A020EDB6A030EDB6A090EDB6A070E5F
:1060E000966E0F01010E1F6F0F01206B929292941A
:1060F0008082810ED56EC70ED56EF29497EC48F073
:10610000050E006E8F0E016E026A00C0E6FFE66E9D
:1061100002C0E6FF800EE66E000EE66E9EEC4AF0D0
:10612000036E050EE15C02E2E16AE552E16E0350A6
:10613000800EE66E000EE66EEAEC48F0E552E5529F
:10614000E80EE66E8E0EE66EF10EE66E8E0EE66ED2
:10615000FD0E006E8E0E016E026A00C0E6FFE66E56
:1061600002C0E6FF800EE66E000EE66E9EEC4AF080
:10617000036E090EE15C02E2E16AE552E16E035052
:10618000800EE66E000EE66EEAEC48F0E552E5524F
:10619000010EE66EE66AD70E006E8E0E016E026A82
:1061A00000C0E6FFE66E02C0E6FF800EE66E000E5F
:1061B000E66E9EEC4AF0036E070EE15C02E2E16AD5
:1061C000E552E16E0350800EE66E000EE66EEAECDC
:1061D00048F0E552E552FC50E66EE66ACA0E006EE3
:1061E0008E0E016E026A00C0E6FFE66E02C0E6FF98
:1061F000800EE66E000EE66E9EEC4AF0036E070E11
:10620000E15C02E2E16AE552E16E0350800EE66E67
:10621000000EE66EEAEC48F0E552E5528450E66E78
:10622000E66ABE0E006E8E0E016E026A00C0E6FFC8
:10623000E66E02C0E6FF800EE66E000EE66E9EEC95
:106240004AF0036E070EE15C02E2E16AE552E16E9C
:106250000350800EE66E000EE66EEAEC48F0E55262
:10626000E552070E8414E76E090EE7CFDBFF00014D
:10627000A86BA96BAA6BAB6B90EC4AF0AE0E006EEC
:106280008E0E016E026A00C0E6FFE66E02C0E6FFF7
:10629000800EE66E000EE66E9EEC4AF0036E050E72
:1062A000E15C02E2E16AE552E16E0350800EE66EC7
:1062B000000EE66EEAEC48F0E552E552F40EE66EAA
:1062C000010EE66E33EC4AF0E552E5528084DFECD5
:1062D00035F0F3CFDBF0F3CF00F0016A00BE0168C8
:1062E00000C0E6FF01C0E6FF960E026E8E0E036E42
:1062F000046A02C0E6FFE66E04C0E6FF800EE66EAA
:10630000000EE66E9EEC4AF0056E070EE15C02E2BE
:10631000E16AE552E16E0550800EE66E000EE66E13
:10632000EAEC48F0E552E5520001DB510EE0DBC03B
:1063300000F0016A00BE016800C0E6FF01C0E6FF90
:10634000F7EC38F0E552E552FFD76CEC36F000017F
:10635000FB511CE0090EDBCFE6FFE66A870E006EFC
:106360008E0E016E026A00C0E6FFE66E02C0E6FF16
:10637000E10EE66E000EE66E9EEC4AF0036E070E2E
:10638000E15C02E2E16AE552E16E03500F011F5148
:106390001EE0770E006E8E0E016E026A00C0E6FFF0
:1063A000E66E02C0E6FF800EE66E000EE66E9EEC24
:1063B0004AF0036E050EE15C02E2E16AE552E16E2D
:1063C00003500001020EAF6F0001210E1DD0670EB9
:1063D000006E8E0E016E026A00C0E6FFE66E02C01D
:1063E000E6FF800EE66E000EE66E9EEC4AF0036E4F
:1063F000050EE15C02E2E16AE552E16E0350000144
:10640000010EAF6F0001040EB06F800EE66E000E3D
:10641000E66EEAEC48F0E552E552080EDB6AC3ECA2
:1064200043F0E10EE66E000EE66E1DEC0FF0E55255
:10643000E5520001DC6FE850DB6FDC51E66EE66A86
:10644000E10EE66E000EE66E520E006E8E0E016ECE
:10645000026A00C0E6FFE66E02C0E6FF800EE66E4E
:10646000000EE66E9EEC4AF0036E090EE15C02E25D
:10647000E16AE552E16E0350800EE66E000EE66EB4
:10648000EAEC48F0E552E5520001DB513CE0DBC0AC
:1064900000F0016A00BE016800C0E6FF01C0E6FF2F
:1064A000F7EC38F0E552E5520001FB0528E1070E54
:1064B0008414006E090EDB50005C21E0070E84148A
:1064C000E76E090EE7CFDBFFDBCFE6FFE66A870E5C
:1064D000006E8E0E016E026A00C0E6FFE66E02C01C
:1064E000E6FFE10EE66E000EE66E9EEC4AF0036EED
:1064F000070EE15C02E2E16AE552E16E03505FDB08
:10650000F3CFDBF08ED782A420D0380E006E8E0E33
:10651000016E026A00C0E6FFE66E02C0E6FF800E72
:10652000E66E000EE66E9EEC4AF0036E050EE15C30
:1065300002E2E16AE552E16E0350800EE66E000E63
:10654000E66EEAEC48F0E552E55237EC19F010EC53
:1065500026F0060EDB6A070EDB6A8250020B01E0B2
:10656000D6D0D950060FE96E000EDA20EA6E050E7D
:10657000EE1801E1ED5001E1CAD00001FB0529E16F
:10658000070E8414006E090EDB50005C22E0070E3B
:106590008414E76E090EE7CFDBFFDBCFE6FFE66A88
:1065A000870E006E8E0E016E026A00C0E6FFE66E78
:1065B00002C0E6FFE10EE66E000EE66E9EEC4AF0CB
:1065C000036E070EE15C02E2E16AE552E16E035000
:1065D0009ED00001AD6BAE6B8074CFEC44F0080E22
:1065E000F3CFDBFFDB5009E0080EDB50006E016AE1
:1065F000FF0E001808E1015006E10001000ED880EE
:10660000AD55000EAE550001DB6B0F011F512AE0A6
:10661000080EDB50070802E1BDEC2CF0080EDB048D
:1066200002E139EC29F0080EDB50020802E198EC97
:1066300029F0080EDB50030808E15CEC2AF0060E96
:10664000F3CFDBFF070EF4CFDBFF080EDB500508AE
:1066500032E1BEEC2BF0060EF3CFDBFF070EF4CFDA
:10666000DBFF29D0080EDB50070802E186EC24F09E
:10667000080EDB50020802E140EC1BF0080EDB04C0
:1066800002E17EEC1BF0080EDB50030802E110EC87
:106690001DF0080EDB50040802E109EC24F0080E9E
:1066A000DB50050802E163EC1EF0080EDB50060823
:1066B00002E147EC24F00001A85101E14ED7A851B6
:1066C000E66EE66AA80EE66E000EE66E290E006E15
:1066D0008E0E016E026A00C0E6FFE66E02C0E6FFA3
:1066E000800EE66E000EE66E9EEC4AF0036E090E1A
:1066F000E15C02E2E16AE552E16E0350800EE66E73
:10670000000EE66EEAEC48F0E552E55226D781BC71
:106710001BD0150E006E8E0E016E026A00C0E6FFE1
:10672000E66E02C0E6FF800EE66E000EE66E9EECA0
:106730004AF0036E050EE15C02E2E16AE552E16EA9
:10674000035081BC19D0FDD7030E006E8E0E016E72
:10675000026A00C0E6FFE66E02C0E6FF800EE66E4B
:10676000000EE66E9EEC4AF0036E050EE15C02E25E
:10677000E16AE552E16E0350800EE66E000EE66EB1
:10678000EAEC48F0E552E5528092E80EE66E030E20
:10679000E66E33EC4AF0E552E5528082E80EE66E92
:1067A000030EE66E33EC4AF0E552E5523AD6D9CF05
:1067B000E6FFDACFE6FFE1CFD9FFE2CFDAFFE6521C
:1067C000E652E652E652E652FA0EDBCFE6FFFB0E49
:1067D000DBCFE6FFFC0EDBCFE6FFFD0EDBCFE6FFF7
:1067E000F40E006E8D0E016E026A00C0E6FFE66ECA
:1067F00002C0E6FF800EE66E000EE66E9EEC4AF0EA
:10680000036E090EE15C02E2E16AE552E16E0350BB
:10681000800EE66E000EE66EEAEC48F0E552E552B8
:10682000020EDB6A030EDB6A020EDBCF00F0030E02
:10683000DBCF01F0D890015004E6500E005C000E52
:10684000015801E390D1020EDBCF02F0030EDBCF43
:1068500003F0040ED89002360336E806FBE1FA0E88
:10686000DBCF04F0FB0EDBCF05F003500518E8AEDC
:1068700002D0053404D00450025C0550035801E3F3
:1068800072D1F10E006E8D0E016E026A00C0E6FF3D
:10689000E66E02C0E6FF800EE66E000EE66E9EEC2F
:1068A0004AF0036E050EE15C02E2E16AE552E16E38
:1068B0000350800EE66E000EE66EEAEC48F0E552FC
:1068C000E552DE6ADD6ADECF00F0DDCF01F0D89060
:1068D000015004E6100E005C000E01586BE2020E3F
:1068E000DBCF04F0030EDBCF05F0040ED8900436A6
:1068F0000536E806FBE1DE500424026EDD5005207B
:10690000036EFA0EDBCF06F0FB0EDBCF07F007506D
:106910000318E8AE02D0033404D00250065C0350E2
:10692000075848E3FC0EDBCF02F0FD0EDBCF03F08F
:10693000DE500224006EDD500320016E100E3F6E0B
:10694000406A020EDBCF44F0030EDBCF45F0BDEC16
:106950004BF000503D24E96E01503E20EA6E040EDB
:10696000EFCFDBFFDBCFE6FFE66AEB0E006E8D0EAE
:10697000016E026A00C0E6FFE66E02C0E6FF800E0E
:10698000E66E000EE66E9EEC4AF0036E070EE15CCA
:1069900002E2E16AE552E16E0350800EE66E000EFF
:1069A000E66EEAEC48F0E552E552DF2A010E8BE391
:1069B000DB2A89D7E70E006E8D0E016E026A00C0D9
:1069C000E6FFE66E02C0E6FF800EE66E000EE66EA3
:1069D0009EEC4AF0036E050EE15C02E2E16AE552CC
:1069E000E16E0350800EE66E000EE66EEAEC48F0B3
:1069F000E552E552DE6ADD6ADECF00F0DDCF01F060
:106A0000D890015004E6100E005C000E015801E31E
:106A1000A3D0020EDBCF04F0030EDBCF05F0040E93
:106A2000D89004360536E806FBE1DE500424026EF9
:106A3000DD500520036EFA0EDBCF06F0FB0EDBCF38
:106A400007F007500318E8AE02D0033404D0025018
:106A5000065C0350075801E27FD0FC0EDBCF02F04A
:106A6000FD0EDBCF03F0DE500224006EDD5003206C
:106A7000016E100E3F6E406A020EDBCF44F0030E33
:106A8000DBCF45F0BDEC4BF000503D24E96E0150EA
:106A90003E20EA6EEF50200839E2FC0EDBCF02F018
:106AA000FD0EDBCF03F0DE500224006EDD5003202C
:106AB000016E100E3F6E406A020EDBCF44F0030EF3
:106AC000DBCF45F0BDEC4BF000503D24E96E0150AA
:106AD0003E20EA6EEF50E66EE66AE40E046E8D0E1E
:106AE000056E066A04C0E6FFE66E06C0E6FF800E8D
:106AF000E66E000EE66E9EEC4AF0076E070EE15C55
:106B000002E2E16AE552E16E075018D0E20E006E33
:106B10008D0E016E026A00C0E6FFE66E02C0E6FF5F
:106B2000800EE66E000EE66E9EEC4AF0036E050ED9
:106B3000E15C02E2E16AE552E16E0350800EE66E2E
:106B4000000EE66EEAEC48F0E552E552DF2A010E4F
:106B500001E252D7DB2A50D7020EDB2A030E01E2F4
:106B600063D6DB2A61D6F10E006E8D0E016E026ACD
:106B700000C0E6FFE66E02C0E6FF800EE66E000E85
:106B8000E66E9EEC4AF0036E050EE15C02E2E16AFD
:106B9000E552E16E0350800EE66E000EE66EEAEC02
:106BA00048F0E552E552050EE15C02E2E16AE55289
:106BB000E16EE552E5CFDAFFE7CFD9FF1200D9CF7A
:106BC000E6FFDACFE6FFE1CFD9FFE2CFDAFFE65208
:106BD000E652050EDE6EDD6A0001630EDB6FDECF6E
:106BE00000F0DDCF01F0013466E200500008000E35
:106BF000015461E20001DB515EE0DF06010E01E2BB
:106C0000DB06D70E006E8D0E016E026A00C0E6FF35
:106C1000E66E02C0E6FF800EE66E000EE66E9EECAB
:106C20004AF0036E050EE15C02E2E16AE552E16EB4
:106C30000350800EE66E000EE66EEAEC48F0E55278
:106C4000E552320EE66EE66A33EC4AF0E552E55262
:106C5000B10EE66E000EE66E11EC0AF0E552E5525A
:106C60000001DB6F006E016A00BE016800C0E6FF34
:106C700001C0E6FFC40E026E8D0E036E046A02C0F0
:106C8000E6FFE66E04C0E6FF800EE66E000EE66EDE
:106C90009EEC4AF0056E070EE15C02E2E16AE55205
:106CA000E16E0550800EE66E000EE66EEAEC48F0EE
:106CB000E552E55294D7DBC000F0016A00BE0168DE
:106CC00000C0F3FF01C0F4FFE552E552E552E5CF05
:106CD000DAFFE7CFD9FF1200D9CFE6FFDACFE6FF20
:106CE000E1CFD9FFE2CFDAFF200EE12402E3E16831
:106CF000E652E16EB30E006E8D0E016E026A00C0A8
:106D0000E6FFE66E02C0E6FF800EE66E000EE66E5F
:106D10009EEC4AF0036E050EE15C02E2E16AE55288
:106D2000E16E0350800EE66E000EE66EEAEC48F06F
:106D3000E552E552EF0EE66E000EE66E1DEC0FF02A
:106D4000E552E5520001DC6FE850DB6FDC51E66E86
:106D5000E66AEF0EE66E000EE66E520E006E8E0EC6
:106D6000016E026A00C0E6FFE66E02C0E6FF800E1A
:106D7000E66E000EE66E9EEC4AF0036E090EE15CD4
:106D800002E2E16AE552E16E0350800EE66E000E0B
:106D9000E66EEAEC48F0E552E5520001DB510AE00C
:106DA000DBC000F0016A00BE016800C0F3FF01C053
:106DB000F4FF11D2D9500A0FE66E000EDA20E66E0B
:106DC000E66A010EE66E000EE66E030EE66E35EC28
:106DD00010F0006E060EE15C02E2E16AE552E16E3F
:106DE00000500001DB6F0A0EDBCFE6FF0B0EDBCF9E
:106DF000E6FFA30E006E8D0E016E026A00C0E6FF74
:106E0000E66E02C0E6FF800EE66E000EE66E9EECB9
:106E10004AF0036E070EE15C02E2E16AE552E16EC0
:106E20000350800EE66E000EE66EEAEC48F0E55286
:106E3000E552020EDB6A030EDB6A040EDB6A050E06
:106E4000DB6A060EDB6A070EDB6A060EDBCF00F09C
:106E5000070EDBCF01F0D890015004E60A0E005C6B
:106E6000000E015824E2D9500C0F006E000EDA20FB
:106E7000016E060EDB500024E96E070EDB50012088
:106E8000EA6EEF6AD950160F006E000EDA20016E1E
:106E9000060EDB500024E96E070EDB500120EA6E7F
:106EA000EF6A060EDB2A070ED0E3DB2ACED7DE6AB6
:106EB000DD6ADECF00F0DDCF01F00A0EDBCF02F09D
:106EC0000B0EDBCF03F00250005C0350015801E3CE
:106ED00058D1DECFE9FFDDCFEAFF000EE926030E31
:106EE000EA22EF500D0801E0E0D0D950160FE66E0F
:106EF000000EDA20E66ED9500C0FE66E000EDA2096
:106F0000E66E970E006E8D0E016E026A00C0E6FFFF
:106F1000E66E02C0E6FF800EE66E000EE66E9EECA8
:106F20004AF0036E090EE15C02E2E16AE552E16EAD
:106F30000350800EE66E000EE66EEAEC48F0E55275
:106F4000E552D9500C0FE66E000EDA20E66E910E77
:106F5000006E8D0E016E026A00C0E6FFE66E02C092
:106F6000E6FF75EC49F0036E050EE15C02E2E16AB2
:106F7000E552E16E035000090DE1D950160FE66E9F
:106F8000000EDA20E66EBEEC49F0E552E552F35011
:106F90000F011F6FD9500C0FE66E000EDA20E66E5F
:106FA0008B0E006E8D0E016E026A00C0E6FFE66E6B
:106FB00002C0E6FF75EC49F0036E050EE15C02E2EB
:106FC000E16AE552E16E035000090DE1D950160F58
:106FD000E66E000EDA20E66EBEEC49F0E552E552B0
:106FE000F3500F01206FD9500C0FE66E000EDA201F
:106FF000E66E840E006E8D0E016E026A00C0E6FF22
:10700000E66E02C0E6FF75EC49F0036E050EE15C2A
:1070100002E2E16AE552E16E035000090DE1D95048
:10702000160FE66E000EDA20E66EBEEC49F0E55271
:10703000E552F3500001FB6F060EDB6A070EDB6AB8
:10704000060EDBCF00F0070EDBCF01F0D890015029
:1070500004E60A0E005C000E015824E2D9500C0F21
:10706000006E000EDA20016E060EDB500024E96E81
:10707000070EDB500120EA6EEF6AD950160F006E42
:10708000000EDA20016E060EDB500024E96E070EBA
:10709000DB500120EA6EEF6A060EDB2A070ED0E312
:1070A000DB2ACED7040EDB6A1BD0DECFE9FFDDCFB3
:1070B000EAFF000EE926030EEA22EF500A085BE021
:1070C000DECFE9FFDDCFEAFF000EE926030EEA225C
:1070D000EF5020080CE1010EF36E040EF3CFDBFF3E
:1070E000050EDB6A020EDB6A030EDB6A44D0D95060
:1070F000040FE96E000EDA20EA6EEE50ED100DE09E
:10710000DECFE9FFDDCFEAFF000EE926030EEA221B
:10711000EF50E66ED950160F0CD0DECFE9FFDDCF71
:10712000EAFF000EE926030EEA22EF50E66ED95080
:107130000C0F006E000EDA20016E020EDB500024F0
:10714000E96E030EDB500120EA6EE552E750EF6E68
:10715000020EDBCF00F0030EDBCF01F0D890015020
:1071600004E60A0E005C000E015805E2020EDB2A5E
:10717000030E01E3DB2ADF2A010E01E29AD6DB2AA5
:1071800098D60F012051E66EE66A0F011F51E66E98
:10719000E66A780E006E8D0E016E026A00C0E6FF90
:1071A000E66E02C0E6FF800EE66E000EE66E9EEC16
:1071B0004AF0036E090EE15C02E2E16AE552E16E1B
:1071C0000350800EE66E000EE66EEAEC48F0E552E3
:1071D000E552F36AF46A200EE15C02E2E16AE552EC
:1071E000E16EE552E5CFDAFFE7CFD9FF1200D9CF44
:1071F000E6FFDACFE6FFE1CFD9FFE2CFDAFF8092F8
:10720000E80EE66E030EE66E33EC4AF0E552E55208
:107210008082E80EE66E030EE66E33EC4AF0E5522D
:10722000E552FC0EDBCF00F0DB06FD0EDBCF01F0FC
:1072300001E2DB06005001100EE080922C0EE66E9B
:10724000010EE66E33EC4AF0E552E55280822C0ED8
:10725000E66E010EE1D78092F40EE66E010EE66E48
:1072600033EC4AF0E552E5528082E552E5CFDAFF91
:10727000E7CFD9FF1200D9CFE6FFDACFE6FFE1CFA3
:10728000D9FFE2CFDAFFE652E652D650026E036A29
:10729000D750046E056A3F6A010E406E04C044F088
:1072A00005C045F0BDEC4BF002503D24006E03508C
:1072B0003E2000C0DEFFDD6EF250040B01E0010E47
:1072C000E66EE66ADECFE6FFDDCFE6FF680E006E13
:1072D0008D0E016E026A00C0E6FFE66E02C0E6FF98
:1072E000800EE66E000EE66E9EEC4AF0036E090E0E
:1072F000E15C02E2E16AE552E16E0350800EE66E67
:10730000000EE66EEAEC48F0E552E552F294E552E2
:0E731000E552E552E5CFDAFFE7CFD9FF1200D4
:02731E00CBECB6
:107320003EF0FB0EDBCFF3FFDB06F35000090AE073
:1073300019EC3FF0FA0E84EC3FF0F3E1011CF1E1AF
:10734000010E01D0000EFAEF3EF0CBEC3EF03B0E0A
:10735000E12402E3E168E652E16E010EDB6A020E0F
:10736000DB6AF90EDBCFF6FFFA0EDBCFF7FFFB0E81
:10737000DBCFF8FF0800F550DF6EDF5002E11EEFB3
:107380003EF0250EDF5C02E011EF3EF0030EDB6AFB
:10739000040EDB6A050EDB6A060EDB6A070EDB6A8B
:1073A00033EC3EF02D0EDF5C0CE02B0EDF5C09E0D1
:1073B000200EDF5C06E0230EDF5C03E0300EDF5CB6
:1073C0001AE1DF50300A14E0130A0FE0030A0AE062
:1073D0000B0A05E0060AE4E1030EDB80E1D7030EA9
:1073E000DB82DED7030EDB84DBD7030EDB86D8D748
:1073F000030EDB88D5D72A0EDF5C1BE12FEC3EF0B5
:107400007DEC3EF010E0030EDB803F684068130E19
:10741000DBCF44F0140EDBCF45F0BDEC4BF0040E97
:107420003DC0DBFF03D0130E66EC3EF033EC3EF0C4
:107430000BD0090EDB6AD4EC3EF003E048EC3FF0E1
:10744000FAD7090E66EC3EF0030EDBB0DB982E0E89
:10745000DF5C1BE133EC3EF02A0EDF5C0BE12FEC2E
:107460003EF07DEC3EF003E1130EB8EC3EF033EC61
:107470003EF00BD0090EDB6AD4EC3EF003E048ECA2
:107480003FF0FAD7090EB8EC3EF0680EDF5C07E17A
:1074900033EC3EF0680EDF5C1DE1030E18D0740E75
:1074A000DF5C17E07A0EDF5C14E0480EDF5C06E07C
:1074B000540EDF5C03E05A0EDF5C02E1020E07D0DF
:1074C0006C0EDF5C03E06A0EDF5C04E1010E0BEC86
:1074D0003FF0C9DBDF506E0A01E17FD31E0A01E1F4
:1074E00092D1200A01E18FD13F0A01E149D11A0A64
:1074F00001E146D10D0A01E143D1200A01E140D169
:107500003A0A01E13DD1200A01E13AD1260A01E11E
:1075100035D10D0A01E132D11A0A01E1D9D0200A90
:107520004AE0300A1FE0460A0EE0250A01E083D354
:10753000D950F90FE96EFF0EDA20EA6E010EEE5E09
:10754000000EEE5AEE5A19EC3FF0250EE66E95DB72
:1075500003E1011C01E169D315EC3FF001E26BD3BB
:10756000DB2A69D3080EDB6A040EDB50010806E251
:10757000040EDB04DDEC3EF0DB508BDB080EDB5051
:1075800009E0030EDB50010B05E172DB01E04DD396
:10759000080EDB6A64DBEFCFDFFF8DEC3FF003E129
:1075A000011C01E142D315EC3FF001E3DB2A60DB73
:1075B00001E141D33AD3070EDB5002080FE159EC49
:1075C0003FF0030E20EC3FF00E0EEECFDBFF0F0E70
:1075D000EECFDBFF100EEECFDBFF20D0F70EDBCFC0
:1075E00003F0F80EDBCF04F0020E035E000E045A27
:1075F000F70E03C0DBFFF80E04C0DBFF03C0E9FF9A
:1076000004C0EAFF10EC3FF0026A0E0E00C0DBFF80
:107610000F0E01C0DBFF100E02C0DBFF0E0EDBCF32
:10762000E6FF0F0EDBCFE6FF100EDBCFE6FF99EC97
:1076300049F0E552E552E552130E3EC0DBFF140E51
:107640003FC0DBFF060EDB5005E0130E54EC3FF0AD
:1076500001E26ADB78EC3FF002E2130E37DB3BEC31
:107660003FF006E0040E54EC3FF002E2050E2EDB84
:10767000030EDBB005D0FCDA01E0D7D2080EDB6ADE
:10768000090EDB6A0E0EDBCFF6FF0F0EDBCFF7FF26
:10769000100EDBCFF8FF0800F550DF6EDF5014E06E
:1076A0007EEC3FF011E28DEC3FF003E1011C01E1C3
:1076B000BCD2BBDB01E3DB2A090EDB2AD9500E0F5B
:1076C000E96E000ECBDBE7D7D3DA01E1B4D2ADD25D
:1076D000C6DA110EEECFDBFF120EEDCFDBFF110E7F
:1076E000DBCFE6FF120EDBCFE6FF8BEC49F0E55275
:1076F000E552130EF3CFDBFF140EF4CFDBFF060EC3
:10770000DB5004E0130ED0DB01E20EDB78EC3FF03F
:1077100002E2130EDBDAAFDB05E0040EC5DB02E2AA
:10772000050ED4DA030EDBB005D0A2DA01E07DD27B
:10773000080EDB6A090EDB6A110EDBCFE9FF120EC1
:10774000DBCFEAFFEFCFDFFFDF5014E0D7DB12E241
:10775000E4DB03E1011C01E168D267DB01E3DB2A22
:10776000090EDB2A110EDB2ADBCFE9FF120EE8E35C
:10777000DB2AE6D77DDA01E15ED257D2030EDB8E3B
:10778000070EDB0410E195DB040E5ADB0A0EEECF88
:10779000DBFF0B0EEECFDBFF0C0EEECFDBFF0D0E93
:1077A000EECFDBFF6CD0070EDB5003082CE1030E9D
:1077B000DBAE0DD0B2DA020E76DAEFCF00F0016A5E
:1077C000026A036A00AE39D00168026835D0F70E4C
:1077D000DBCF01F0F80EDBCF02F0020E015E000EEF
:1077E000025AF70E01C0DBFFF80E02C0DBFF01C03A
:1077F000E9FF02C0EAFFEFCF00F00A0E00C0DBFF96
:107800000B0EDB6A38D0070EDB50020809E1030ECD
:10781000DBAE04D059DB02AE10D00ED055DB0DD05C
:10782000030EDBAE12D079DA020E3DDAF9DA026A23
:10783000036A01AE02D002680368E2DA0C0E02C0ED
:10784000DBFF0D0E03C0DBFF1AD0F70EDBCF02F01B
:10785000F80EDBCF03F0020E025E000E035AF70EA5
:1078600002C0DBFFF80E03C0DBFF02C0E9FF03C06C
:10787000EAFFD6DAC5DA0C0EDB6A0D0EDB6A060EFD
:10788000DB5005E1010EF36E050EF3CFDBFF150EA5
:10789000DB6A160EDB6AD950370F006E000EDA2055
:1078A000016E390E00C0DBFF3A0E01C0DBFF380E5F
:1078B000DB6A080EDB6A0A0EAEDADF50780A12E0E5
:1078C000200A10E0280A0CE0200A0AE03F0A06E03D
:1078D0000D0A02E0200A08E1020E05D0080E03D0CE
:1078E000080EDF26100E97DA030EDBBE02D0DB9205
:1078F000DB94DB50800B24E08ADAD890030EEB5047
:10790000000A08E6000EEE5C000EEE58000EEE587F
:10791000000EEE5815E213DA426843684468456881
:1079200085EC4BF00A0E39C0DBFF0B0E3AC0DBFFD3
:107930000C0E3BC0DBFF0D0E3CC0DBFF2D0E08D054
:10794000030EDBA202D02B0E03D0DBA408D0200E46
:10795000F36E170EF3CFDBFF150EDB2A02D0170EE6
:10796000DB6A050EDB5003E1B7D901E189D0E60EF1
:10797000006E980E016E000E026E070EDBCF03F054
:10798000046A056A066A03C042F004C043F005C0F9
:1079900044F006C045F0D3D9EAEC4BF0005039244E
:1079A000F36E01503A20F46E02503B20F86EF4CF93
:1079B000F7FFF3CFF6FF0800090EF5CFDBFF580EF7
:1079C000DF5C0FE1610EF36E090E7BD90AE3200E36
:1079D000006E090EDBCFE7FF0050E75E090EE7CF30
:1079E000DBFF070EDBCF00F0016A026A036A0FDAE1
:1079F00000C042F001C043F002C044F003C045F0B3
:107A0000EECF3DF0EECF3EF0EECF3FF0EFCF40F0C7
:107A1000EAEC4BF040C0EDFF3FC0EDFF3EC0EDFF94
:107A20003DC0EFFF390EDBCFE9FFDB063A0EDBCFBF
:107A3000EAFF01E2DB06090EDBCFEFFF150EDB2AC2
:107A40004BD995E1030EDBA61DD06F0EDF5C06E17E
:107A5000C1D918E3150EDB285BDA14D0780EDF5C91
:107A600009E0580EDF5C06E0620EDF5C03E0420EC8
:107A7000DF5C08E1020EF36E160EF3CFDBFF02D0DF
:107A8000150EDB6A030EDB50100B0EE0040EDBCF8D
:107A900000F0050EDB50D880005406E2060EDB50E5
:107AA00003E1040EDB5034DA95D90AE2050EDBCF90
:107AB000E7FF150EDB50E75E050EE7CFDBFF02D0D8
:107AC000050EDB6A040EDBCF00F0160E45D9D88018
:107AD000005414E2160EDBCFE6FF150EDBCFE6FFF7
:107AE000040EDBCFE6FF050EDB50E552E75CE55206
:107AF000D880E754E552D880E7545FD9030EDB50B5
:107B0000010B0BE1080EDB5008E0B2D801E08DD08C
:107B1000080EDB50BED8080EDB6A170EDB5007E0FC
:107B200088D9170EF1D903E1011C01E17ED0160EB0
:107B3000DB5016E07ED9300EE66E9FD802E1011CC4
:107B400074E077D9DFCFE6FF43EC4BF0E552E55226
:107B5000E552F4CF01F00001F31C02E1011C65E0E5
:107B6000050EDBCF00F0160EDB50D880005409E282
:107B7000050EDBCFE7FF160EDB50E75E050EE7CF05
:107B8000DBFF300EE66E050ECBD94FE1390EDB2A56
:107B9000DBCFE9FF3A0E01E3DB2ADBCFEAFF090E78
:107BA000EFCFDBFFDB500EE044D9090EADD902E187
:107BB000011C3BE0390EDB2ADBCFE9FF3A0EEDE397
:107BC000DB2AEBD755D831E1160EDBCFE6FF080EE6
:107BD000C3D8E552E7245DD82ED0070EDB50030A48
:107BE0001CE0010A14E0030A07E07BD9DBCFEEFFBB
:107BF000020EDBCFEDFF1FD0F5D8056A03AE02D031
:107C0000046805682CD8BCD805C0EEFF14D0EAD8AB
:107C100003BE046824D8B4D80ED063D9DBCFEFFFFD
:107C20000AD07BD905E1011C03E1F368F46810D0A8
:107C3000FCD801E3DB2A79D9BAEF39F0010EDBCFAA
:107C400000F0020EDBCF01F000C0F3FF01C0F4FF33
:107C50003B0EE15C02E2E16AE552E16ECBD029D94C
:107C6000020E20EF3FF061D90800F550DF6E1200E0
:107C7000200EE66E080E90EF3FF043EC4BF0E5521D
:107C8000E552E552F3CF00F0F4CF01F00001F31C10
:107C90001200006E016AD950010F4DD90050EE2636
:107CA0000150ED221200045E000E055AF70E04C0CA
:107CB000DBFFF80E05C0DBFF04C0E9FF05C0EAFFEB
:107CC0001200DBCFF4FFF350F45C1200DB50E76EE0
:107CD000040EE7CFDBFF12000A0EDBCF00F00B0E25
:107CE000DBCF01F00C0EDBCF02F00D0EDBCF03F08B
:107CF00000500110021003101200130EEECFDBFF34
:107D0000140EEDCFDBFF130EDBCF00F0140EDBCF34
:107D100001F00001800E01141200F70EDBCF04F019
:107D2000F80EDBCF05F01200050EDB50E66ED950E1
:107D3000130F01D9E552E750EE6EED6A12000A0EFC
:107D4000DBCF3DF00B0EDBCF3EF00C0EDBCF3FF078
:107D50000D0EDBCF40F01200DBCFE6FF150EDBCFC0
:107D6000E6FF050EDB50E552E724E552E72412005A
:107D7000DB50CED8010EF36E060EF3CFDBFF120000
:107D8000EE50EFCFEAFFE96E02C0EEFF03C0EEFF58
:107D900004C0EEFF1200D9CFE6FFDACFE6FFE1CF55
:107DA000D9FFE2CFDAFF1200DFCFE6FFE66A25EC6B
:107DB0004CF0E552E552F3501200E76E080EE7CFA3
:107DC000DBFF1200EECF00F0EECF01F0EFCF02F0BC
:107DD000036A1200050EDBCF00F0150EDB50D880D1
:107DE00000541200010EDBCF02F0020EDBCF03F0D5
:107DF000046A1200E552E5CFDAFFE7CFD9FF12009F
:107E00000A0E00C0DBFF0B0E01C0DBFF1200D950D1
:107E10000A0F9BEF3FF0F36E070EF3CFDBFF12006C
:107E2000EECF00F0EFCF01F01200010EDB2A020EC0
:107E30001200FC0EDBCFE6FFFD0EDBCFE6FF1200EB
:107E4000005E000E015AF70E00C0DBFFF80E01C005
:107E5000DBFF00C0E9FF01C0EAFF1200DA20EA6E92
:107E6000EF2AEECFF6FF000EEF22EECFF7FFEF2264
:107E7000EECFF8FF1200040EDBCFE6FF130EDB504F
:107E8000E552E75C9ADFDB5004DF060EDB501200A0
:107E9000090EDB500A0DF350DF24D00FE76E090EF8
:107EA000E7CFDBFF33EF3EF0DB50F36E050E61EF03
:107EB0003EF0F70EDBCF00F0F80EDBCF01F0120042
:107EC000DFCFE6FF3DEF3EF028DF030EECDEE2EF12
:107ED0003EF08FEC39F0E552E552E552E5520009EB
:107EE0001200BDDEEE50EFCFEAFFE96E010E120088
:107EF000130EDB50F36E040E61EF3EF0040EDB5008
:107F0000F36E090E61EF3EF0DBCFE6FF3DEF3EF092
:107F1000E76E050EE7CFDBFF12008BDF60EF3FF06F
:107F2000DBCFE6FF86DF69EF3FF0D950F90FE96E4E
:107F3000FF0E2EEF3FF0E96E000EDA20EA6E12001F
:107F4000D9CFE6FFDACFE6FFE1CFD9FFE2CFDAFF04
:107F5000FD0EDB5003E0C66A010E02D0C66A020EB7
:107F6000C66E400EC76EC68AE552E5CFDAFFE7CF90
:107F7000D9FF1200D9CFE6FFDACFE6FFE1CFD9FF74
:107F8000E2CFDAFFE652E652500EDE6EDD6AD9CF5E
:107F9000E9FFDACFEAFFEE06000EED5AEECF00F071
:107FA000EDCF01F000500110F2E1E552E552E5524B
:107FB000E5CFDAFFE7CFD9FF1200D9CFE6FFDACF5E
:107FC000E6FFE1CFD9FFE2CFDAFFFD0EDB50C96E4D
:107FD000C7B0FED7C7A0FED7FD0EC9CFDBFFE55265
:107FE000E5CFDAFFE7CFD9FF1200C968C7B0FED7E7
:107FF000C7A0FED7C9501200D9CFE6FFDACFE6FFFF
:10800000E1CFD9FFE2CFDAFFE652E652FD0EDBAE5A
:1080100018D0FD0EDB9EE66AE66AE66AE66A770E2F
:10802000E66EEADF006E050EE15C02E2E16AE5520F
:10803000E16E0050E76E010EE7CFDBFFDB50010879
:1080400074E38280D2DF8290D0DFFD0EDBCFE6FFCB
:10805000B4DFE552F90EDBCF00F0FA0EDBCF01F012
:10806000FB0EDBCF02F0FC0EDBCF03F0180ED89036
:108070000332023201320032E806F9E10050E66EC6
:108080009CDFE552F90EDBCF00F0FA0EDBCF01F0FA
:10809000FB0EDBCF02F0FC0EDBCF03F0100ED8900E
:1080A0000332023201320032E806F9E10050E66E96
:1080B00084DFE552F90EDBCF00F0FA0EDBCF01F0E2
:1080C000FB0EDBCF02F0FC0EDBCF03F0080ED890E6
:1080D0000332023201320032E806F9E10050E66E66
:1080E0006CDFE552F90EDBCFE6FF67DFE552010EEC
:1080F000DF6EFD0EDB50400802E1950EDF6EFD0ED7
:10810000DB50480802E1870EDF6EDFCFE6FF55DF68
:10811000E5520A0EDF6E69DFE76E010EE7CFDBFF87
:10812000DB50800B02E0DF06F6E1010EDB50E5528A
:10813000E552E552E5CFDAFFE7CFD9FF1200D9CFFC
:10814000E6FFDACFE6FFE1CFD9FFE2CFDAFF090E93
:10815000E12402E3E168E652E16EE66AF1DEE5520F
:10816000720ED36E0001FC5113E08250010B10E13E
:10817000E66AE66AE66AE66A000EE66EE66A1BDA18
:10818000006E060EE15C02E2E16AE552E16E00502B
:1081900082800A0EDF6EDF5003E027DFDF06FBD7A9
:1081A000020EDB6AE66AE66AE66AE66A400EE66E98
:1081B00023DF006E050EE15C02E2E16AE552E16E4A
:1081C0000050010801E008D1AA0EE66E010EE66E2D
:1081D000E66AE66A480EE66E0FDF006E050EE15CA9
:1081E00002E2E16AE552E16E0050010801E08DD043
:1081F000DF6A040EDF5C14E2F8DEE66ED950030F8E
:10820000006E000EDA20016EDF500F010024E96ECF
:10821000000E0120EA6EE552E750EF6EDF2AE9D743
:10822000050EDB0401E0D8D0060EDB50AA0801E001
:10823000D3D0100EF36E070EF3CFDBFF270EF36ED5
:10824000080EF3CFDBFFD950070FE96E000EDA20DE
:10825000EA6EEE50ED1019E0E66AE66AE66A400E54
:10826000E66EE90EE66EC8DE006E050EE15C02E227
:10827000E16AE552E16E0050000907E07BDE070E7F
:10828000DB06080EE0E2DB06DED7D950070FE96E09
:10829000000EDA20EA6EEE50ED1001E19DD0E66AA4
:1082A000E66AE66AE66A7A0EE66EA6DE006E050EFD
:1082B000E15C02E2E16AE552E16E0050000901E092
:1082C0008BD0DF6A040EDF5C14E28FDEE66ED950DD
:1082D000030F006E000EDA20016EDF500F01002444
:1082E000E96E000E0120EA6EE552E750EF6EDF2ADC
:1082F000E9D7030EDB50400B02E00C0E01D0040E58
:10830000E76E020EE7CFDBFF67D0E66AE66AE66A51
:10831000E66AE90EE66E70DE006E050EE15C02E2D2
:10832000E16AE552E16E0050010805E3020EDB6EE2
:10833000DE52E90E07D0010EF36E020EF3CFDBFF23
:10834000DE52410EDD6E100EF36E070EF3CFDBFF33
:10835000270EF36E080EF3CFDBFFD950070FE96E3F
:10836000000EDA20EA6EEE50ED1019E0E66AE66AD9
:10837000E66AE66A010EDBCFE6FF3EDE006E050E22
:10838000E15C02E2E16AE552E16E0050000907E0BB
:10839000F1DD070EDB06080EE0E2DB06DED7D95082
:1083A000070FE96E000EDA20EA6EEE50ED1012E0D3
:1083B000E66A020EE66EE66AE66A500EE66E1CDEBD
:1083C000006E050EE15C02E2E16AE552E16E0050EA
:1083D000000902E0020EDB6A020EDBCFFCF08280B5
:1083E00004DE010EE66EACDDE552D36A020EDB5010
:1083F00002E0000E01D0010E006E090EE15C02E207
:10840000E16AE552E16E0050E552E5CFDAFFE7CFD1
:10841000D9FF1200D9CFE6FFDACFE6FFE1CFD9FFCF
:10842000E2CFDAFFE652E652E652E6520001FCB72E
:1084300012D0D950F80FE96EFF0EDA20EA6E090E5D
:10844000E76ED890EF36010EEB36020EEB36030ED8
:10845000EB36E706F6E1010EDF6ED950F80FE96E54
:10846000FF0EDA20EA6EEECFE6FFEECFE6FFEECFAC
:10847000E6FFEFCFE6FF510EE66EBEDD006E050EA5
:10848000E15C02E2E16AE552E16E0050000901E0C0
:1084900081D0400EF36E020EF3CFDBFF9C0EF36E25
:1084A000030EF3CFDBFFA1DDE76E010EE7CFDBFFAD
:1084B000DB50FF080CE1020EDB06DBCF00F0030E01
:1084C00001E2DB06DBCF01F000500110ECE1010E10
:1084D000DB50FE085FE1F60EDBCF02F0F70EDBCFDC
:1084E00003F0020ED88002560356F40EDB50025CF5
:1084F000006EF50EDB500358016E020E00C0DBFF6C
:10850000030E01C0DBFFD950F60FE96EFF0EDA2033
:10851000EA6EEE50ED100DE068DDF60EDB06DBCF07
:1085200000F0F70E01E2DB06DBCF01F00050011096
:10853000F3E1D950FC0FE96EFF0EDA20EA6EEE503F
:10854000ED101AE052DDE66EFC0EDBCFE9FFDB2A10
:10855000FD0EDBCFEAFF01E3DB2AE552E750EF6EC9
:10856000F40EDB06DBCF00F0F50E01E2DB06DBCF1D
:1085700001F000500110E6E138DD020EDB06DBCF32
:1085800000F0030E01E2DB06DBCF01F0005001102A
:10859000F3E1DF6A828029DDDF50006E040EE15CCA
:1085A00002E2E16AE552E16E0050E552E5CFDAFF02
:1085B000E7CFD9FF1200D9CFE6FFDACFE6FFE1CF50
:1085C000D9FFE2CFDAFFE652E652E652010EDF6E45
:1085D000D950FC0FE96EFF0EDA20EA6EEE50ED1076
:1085E00030E0F80EDBCF3FF0F90EDBCF40F0DE528B
:1085F0003FC0DEFF40C0DDFFDD52D950010FE96E04
:10860000000EDA20EA6EEE50ED1067E00001FD5139
:10861000FE1163E0FC0EDBCFE9FFDB2AFD0EDBCFB2
:10862000EAFF01E3DB2AEF50E66EC7DCE55200010A
:10863000FD07000EFE5B010EDB06020EDEE2DB062E
:10864000DCD7F80EDBCF00F0F90EDBCF01F0FA0E2D
:10865000DBCF02F0FB0EDBCF03F000500110021065
:1086600003103DE00001FCB712D0D950F80FE96EBD
:10867000FF0EDA20EA6E090EE76ED890EF36010E93
:10868000EB36020EEB36030EEB36E706F6E1D95079
:10869000F80FE96EFF0EDA20EA6EEECFE6FFEECFBE
:1086A000E6FFEECFE6FFEFCFE6FF580EE66EA4DC66
:1086B000006E050EE15C02E2E16AE552E16E0050F7
:1086C000000957E1E66879DCE552FE0EE66E75DCDE
:1086D000E5520001FD6B020EFE6FDF6A4AD0020E0A
:1086E0000001016AFD25006EFE510122010E00C04D
:1086F000DBFF020E01C0DBFF010EDBCF00F0DB066B
:10870000020EDBCF01F001E2DB060050011004E0B5
:10871000E66A53DCE552F0D768DC1F0B050827E159
:10872000880EF36E010EF3CFDBFF130EF36E020E15
:10873000F3CFDBFF5ADCFF0810E0D950010FE96EE0
:10874000000EDA20EA6EEE50ED1007E013DC010EA9
:10875000DB06020EEFE2DB06EDD7D950010FE96E22
:10876000000EDA20EA6EEE50ED1001E0DF6A828042
:108770003CDCDF50E552E552E552E552E5CFDAFF49
:06878000E7CFD9FF120053
:0A87860081868A908A928A9493807B
:10879000938293849568938C938E9388938A93861F
:1087A00092900001AD6BAE6B1F6A206AFF0E1F5CDA
:1087B000000E20580BE2000E1F24E96E010E20204F
:1087C000EA6EEF6A1F2A000E2022F0D71F6A206A85
:1087D000FF0E1F5C000E20580BE2000E1F24E96EF6
:1087E000020E2020EA6EEF6A1F2A000E2022F0D728
:1087F0002F6A1200D9CFE6FFDACFE6FFE1CFD9FF2B
:10880000E2CFDAFF2C6A216A226A080E8A148A6E85
:1088100093868A908A928A948A989380938293848A
:1088200093889568630E2C5C01E1AAD08150400BBF
:1088300001E1A6D0A00E236E860E246E010E256ED9
:10884000266A2C50620A01E174D0640A62E0030ACD
:1088500057E0010A4FE0070A45E0020A22E0030A56
:1088600020E0020ADFE18150020B61E08150040B3D
:108870005EE023C000F024C001F025C002F026C055
:1088800003F02306000E245A255A265AD880005495
:10889000000E0154000E0254000E0354C3E3620E96
:1088A0006DD0FC0EDBCF00F0FD0EDBCF01F000063B
:1088B000000E015A0050211807E10150221804E16E
:1088C000020E1E1401E0939A000E2124E96E020E9E
:1088D0002220EA6EEF1C8C6E212A000E2222956A5D
:1088E000030E0AD081A202D0040E2C6EF2A49AD7F5
:1088F000040E0DD09390050E2C6ED66AF29492D78A
:1089000081A402D0060E2C6EF2A48CD7060E2B6E1C
:1089100089D79568938A9380FC0EDBCF00F0FD0E1B
:10892000DBCF01F00050215C0150225826E2010EFD
:1089300025D0220EE66E8F0EE66E280E006E8F0E8C
:10894000016E026A00C0E6FFE66E02C0E6FF800E1E
:10895000E66E000EE66E9EEC4AF0036E070EE15CDA
:1089600002E2E16AE552E16E0350800EE66E000E0F
:10897000E66EEAEC48F0E552E552630E2C6E52D7F3
:108980009380938293849388938A9568F70E9310CB
:10899000936EE552E5CFDAFFE7CFD9FF1200D9CFCA
:1089A000E6FFDACFE6FFE1CFD9FFE2CFDAFFE6520A
:1089B000E652DF6AD00E276E070E286E296A2A6AF1
:1089C0000001AD6BAE6B010EDB6A8A6A93868A90FA
:1089D0008A928A94819281949380939293949568D9
:1089E0002B6AE66AE66EE66A000EE66E010EE66E39
:1089F0005BEC49F0006E050EE15C02E2E16AE552D3
:108A0000E16E0050630E2B5C01E1C5D00001000E49
:108A1000AD5D010EAE5903E28150400B02E1090E3B
:108A20002B6E2B50090A01E1B1D0030A01E1AAD053
:108A30000C0A01E192D0030A45E0010A3FE0070A6F
:108A400016E0010A0CE0030A05E0010ADBE193925B
:108A5000939481D09382D66AF294020E9AD081B018
:108A600002D0030E2B6EF2A4CDD70A0E92D0D00EF8
:108A7000276E070E286E296A2A6A9392831CE66E77
:108A8000000EAD25E96E010EAE21EA6EE552E7500B
:108A9000EF6E8150200B01E0010E2D6E8150100B06
:108AA00001E0010E2E6EAD2B000EAE230A0E236EDA
:108AB000246A256A266A9384040E6BD081A0A2D70B
:108AC000050E67D093940F011F5118E02F50E66EEA
:108AD0002E5002E0000E01D0010EE66EADC0E9FF9F
:108AE000AEC0EAFFE906000EEA5A000EE926010EC2
:108AF000EA22EF50E66EA1EC26F017D02F50E66E7A
:108B00002E5002E0000E01D0010EE66EADC0E9FF6E
:108B1000AEC0EAFFE906000EEA5A000EE926010E91
:108B2000EA22EF50E66E40EC19F0E552E552E552CC
:108B3000010EF3CFDBFFDB5027E12D500CE1060ED9
:108B40002B6EE80E236E030E246E256A266ADE5213
:108B5000FE0EDD6E57D7010E1CD0938481AA02D081
:108B6000090E2B6E2306000E245A255A265AD88049
:108B70002354000E2454000E2554000E265401E206
:108B800041D702D0010EDF6E090E03D09392939469
:108B9000630E2B6E37D72E5030E1ADC0E9FFAEC06B
:108BA000EAFFE906000EEA5A000EE926010EEA2263
:108BB000EF50600822E1ADC0E9FFAEC0EAFF020E4F
:108BC000E95E000EEA5A000EE926010EEA22EF5095
:108BD0005F0813E1020E1E101E6EAFC000F2B0C09F
:108BE00001F2020EE66EE66A05DEE552E552FD0E82
:108BF0001E141E6E0001AD6BAE6B0001000ED8801E
:108C0000AD55000EAE55DF5003E0F368F46A07D0AF
:108C1000010EDB50006E016AF36E01C0F4FFE552F5
:108C2000E552E552E5CFDAFFE7CFD9FF1200819C8C
:108C3000939CA00E236E860E246E010E256E266A6E
:108C4000235024102510261006E02306000E245A77
:108C5000255A265AF5D7818C938CA00E236E860E4A
:108C6000246E010E256E266A23502410251026102E
:108C700006E02306000E245A255A265AF5D712007C
:108C8000D9CFE6FFDACFE6FFE1CFD9FFE2CFDAFFB7
:108C9000FD0EDB0403E19396819602D093868186D4
:108CA000E552E5CFDAFFE7CFD9FF1200D9CFE6FFD3
:108CB000DACFE6FFE1CFD9FFE2CFDAFFE652E652A4
:108CC000D650026E036AD750046E056A3F6A010EE1
:108CD000406E04C044F005C045F0BDEC4BF00250BE
:108CE0003D24006E03503E2000C0DEFFDD6EF250DA
:108CF000040B01E0010EE66EE66ADECFE6FFDDCF93
:108D0000E6FFFD0EDBCF00F0016A00BE016800C087
:108D1000E6FF01C0E6FF170E026E8F0E036E046AB7
:108D200002C0E6FFE66E04C0E6FF800EE66E000EAF
:108D3000E66E9EEC4AF0056E0B0EE15C02E2E16A23
:108D4000E552E16E0550800EE66E000EE66EEAEC2E
:108D500048F0E552E552F294E552E552E552E5CF8E
:088D6000DAFFE7CFD9FF120092
:088D68000D0A5469636B733AB4
:108D700025752025640D0A000D0A503A256420440B
:108D80003A25640044534B53454C004445425547F3
:108D90000050524F544F000D0A4B3A257320563A5B
:108DA0002573000D0A526561642025642062797480
:108DB0006573000D0A52656164696E6720636F6EAA
:108DC000666967000D0A4D6F756E74207265747563
:108DD000726E73202558000D0A4D6F756E74696EA2
:108DE00067002E00256300207C20002025303258AB
:108DF000000D0A000D0A44756D7020255820255875
:108E00000D0A000D0A0D0A4F6F70732E204E6F2051
:108E100063617264000D0A0D0A496E7465726661C1
:108E2000636520636C656172000D0A456467653A8D
:108E300020257320202564000D0A43617264206997
:108E4000732077726974652070726F7465637465DE
:108E500064000D0A4F70656E20257320726574756D
:108E6000726E73202558000D0A416D69676F2039B5
:108E7000313231440D0A000D0A53532F3830203956
:108E80003133344C0D0A002F6C69666461746125BE
:108E9000642E62696E000D0A0D0A53445F6D6F7592
:108EA0006E742072657475726E73202564000D0AED
:108EB00048617264776172652050500D0A000D0A96
:108EC000504F5254453A202558000D0A53544B50E8
:108ED00054523A202558000D0A534420535049203B
:108EE0004449563A2025640032313A32383A35380E
:108EF000004E6F762031382032303136000D0A2591
:108F000053202553000D0A0D0A48504469736B2005
:108F10007620302E3233000D0A25643A257520253F
:108F200064007B4552527D002553000D0A414D3AA5
:108F300020496E6372656D656E743A202564202544
:108F4000642025642025642C20000D0A414D3A43FD
:108F50006C656172000D0A414D3A57616B65757021
:108F6000000D0A414D3A44534A000D0A414D3A4220
:108F700075666620777220256C642062797465734B
:108F8000207278000D0A436C6F73696E67207772E8
:108F9000206661696C202564000D0A57726974654A
:108FA000206661696C202564000A002E002563009C
:108FB000207C20002025303258000D0A000D0A5276
:108FC00064206576656E20736563746F723A202540
:108FD0006C6420617420256C58202564000D0A52B1
:108FE00064206F646420736563746F723A20256C2B
:108FF0006420617420256C58202564000D0A414DC1
:109000003A4275666620777220632F682F733A2084
:1090100025642F25642F256420733A256C64000D88
:109020000A20256C642062797465732073656E7400
:10903000000D0A526561642072657475726E73204A
:1090400025582C202564206279746573207265612F
:1090500064000D0A414D3A427566662072642063D1
:109060002F682F733A2025642F25642F25642073E1
:109070003A256C6420000D0A5365656B20746F20DF
:10908000256C64206661696C6564202564000D0AA6
:109090005365656B696E6720746F20256C642028AA
:1090A000256C5829000D0A414D3A205365656B3AED
:1090B0002025642025642025642025642C20733A13
:1090C000256C64000D0A414D3A53656E642073743B
:1090D00061747573005B4D4C415D005B4D54415DA7
:1090E000007B25752025647D5B253032585D007B33
:1090F0005425752025647D5B253032585D007B4CFE
:1091000025752025647D5B253032585D000D0A727F
:10911000633D2564000D0A4D617820566563746FC8
:0D9120007220256C642028256C5829200041
:02912E000C0E25
:10913000AF6EB06AB896AC98AB8EAB88AB9A9D9880
:109140009D9AD08E9F8AF28EAC90AB9CAC9AAC8AE2
:10915000AC9404018191806B1200D9CFE6FFDACF85
:10916000E6FFE1CFD9FFE2CFDAFFACA2FED7FD0EDA
:10917000DBCFE6FF0EEC4CF0E552E552E5CFDAFF2F
:10918000E7CFD9FF12009EBA03D0040007D8FBD75F
:10919000AE5000D012009EBA010C000CD9CFE6FFF1
:1091A000DACFE6FFE1CFD9FFE2CFDAFFE652ABA29A
:1091B00004D0AC9AAC8AAB98AB88ABA404D0AE50C8
:1091C000DF6EAC9AAC8AE552E552E5CFDAFFE7CF25
:1091D000D9FF1200D9CFE6FFDACFE6FFE1CFD9FF02
:1091E000E2CFDAFF0401826B836BFC0EDBCFE9FF79
:1091F000FD0EDBCFEAFFEF5014E0FC0EDBCFE9FF02
:10920000FD0EDBCFEAFFEF50E66EA7DFE552FC0E66
:10921000DB2AFD0E01E3DB2A0401822B000E8323EF
:10922000E4D7280E83AF02D0D89003D0825D000E21
:10923000835910E3230EE66E90DFE5524F0EE66E83
:109240008CDFE552460EE66E88DFE552230EE66EB1
:1092500084DFE552E552E5CFDAFFE7CFD9FF120010
:10926000D9CFE6FFDACFE6FFFA0EE3CFD9FFFB0E48
:10927000E3CFDAFFFC0EE3CFE9FFFD0EE3CFEAFF19
:10928000E9CFF3FFEACFF4FFF80EE35003E1F90E64
:10929000E35008E0F80EE30602E2F90EE306DECF43
:1092A000EEFFF2D7FF0EE3CFDAFFE552FF0EE3CF7A
:1092B000D9FFE5521200FE0EE3CFE9FFFF0EE3CF28
:1092C000EAFFE9CFF3FFEACFF4FFFB0EE35003E13F
:1092D000FC0EE35009E0FB0EE30602E2FC0EE3069F
:1092E000FD0EE350EE6EF1D71200FD0EE3CFF6FF58
:1092F000FE0EE3CFF7FFFF0EE3CFF8FFFB0EE3CF49
:10930000E9FFFC0EE3CFEAFFEE500900F55C02E155
:10931000F566FAD71200FE0EE3CFE9FFFF0EE3CFAA
:10932000EAFFF36AF46AEE5203E0F34AF42AFBD749
:109330001200FF0EE3CFF8FFE552FF0EE3CFF7FF79
:10934000E552FF0EE3CFF6FFE552E66AE66AE66A0B
:109350000900F55209E0FD0EE32A05E1FE0EE32ABD
:1093600002E1FF0EE32AF4D7FD0EE3CF3EF0FE0E3E
:0C937000E3CF3FF0FF0EE3CF40F012000F
:04937C00FF0EE3CF2E
:10938000EAFFE552FF0EE3CFE9FFE552E66AE66A3F
:10939000D9CFE6FFDACFE6FFFC0EE124D96EFF0E4F
:1093A000E220DA6EE66AE66AE66A200EEF5C06E024
:1093B000090EEF5C03E0EF6603D03FD0EE50F5D727
:1093C0002D0EEF5C03E1FF0EE32A03D02B0EEF5CC2
:1093D00001E1EE502F0EEF6424D03A0EEF6021D061
:1093E000D890F90EE336FA0EE336FD0EDECFE3FF3A
:1093F000FE0EDDCFE3FFD890F90EE336FA0EE3362A
:10940000D890F90EE336FA0EE336FD0EE350DE2671
:10941000FE0EE350DD22300EEE5CDE26000EDD2275
:10942000D9D7FF0EE3CFE8FFE85207E0F90EE31EBD
:10943000E32AFA0ED8B4E306E31EE552E552E552FC
:10944000FF0EE3CFDAFFE552FF0EE3CFD9FFE5527F
:10945000E1CFE9FFE2CFEAFFED52ED52EECFF3FFAD
:06946000EFCFF4FF120043
:0A946600D9CFE6FFDACFE6FFE1CF31
:10947000D9FFE2CFDAFFE652E652DE6ADD6ADECFDE
:1094800000F0DDCF01F0FC0EDBCF02F0FD0EDBCFF4
:1094900003F00250005C035001580AE2080EE66E29
:1094A00037EC4CF0E552DF2A010EE9E3DB2AE7D77F
:1094B000E552E552E552E5CFDAFFE7CFD9FF1200DA
:1094C000D9CFE6FFDACFE6FFE1CFD9FFE2CFDAFF6F
:1094D000E652E652DE6ADD6ADECF00F0DDCF01F053
:1094E000FC0EDBCF02F0FD0EDBCF03F00250005C80
:1094F000035001580DE200000000000000000000D1
:10950000000000000000DF2A010E01E3DB2AE4D79F
:10951000E552E552E552E5CFDAFFE7CFD9FF120079
:10952000C2900F0EC16E070EB46ED36A4F0EC86E96
:0C953000946A948894829484826A1200E9
:04953C00D9CFE6FF9E
:10954000DACFE6FFE1CFD9FFE2CFDAFFE652E6520B
:10955000E652E652D950F90F006EFF0EDA20016E86
:10956000020E00C0DBFF030E01C0DBFF020EDBCFEB
:10957000E6FF030EDBCFE6FFF90EDBCFE6FFFA0EC8
:10958000DBCFE6FFFB0EDBCFE6FFD950FC0FE66E2C
:10959000FF0EDA20E66EA5EC39F0006E070EE15CF6
:1095A00002E2E16AE552E16E0050F3CFDEFFF4CF54
:1095B000DDFFFC0EDBCFE9FFFD0EDBCFEAFFEF6A3C
:1095C000DECF00F0DDCF01F000C0F3FF01C0F4FFFB
:1095D000040EE15C02E2E16AE552E16EE552E5CF9C
:0895E000DAFFE7CFD9FF12000A
:0895E800060EF66E000EF76E90
:1095F000000EF86E0F010900F5501A6F0900F550C2
:109600001B6F03E11A6701D03DD00900F550156FBB
:109610000900F550166F0900F550176F0900090091
:10962000F550E96E0900F550EA6E090009000900DD
:10963000F550186F0900F550196F09000900F6CFB1
:109640001CFFF7CF1DFFF8CF1EFF15CFF6FF16CF7B
:10965000F7FF17CFF8FF0F01185302E1195307E086
:109660000900F550EE6E1807F8E21907F9D71CCF7C
:10967000F6FF1DCFF7FF1ECFF8FF0F011A07000EF0
:069680001B5BBFD71200C6
:0A968600D9CFE6FFDACFE6FFE1CF0F
:10969000D9FFE2CFDAFFFB0EDBCF00F0FC0EDBCF11
:1096A00001F00001800E01141AE1FB0EDBCFE9FF8F
:1096B000FC0EDBCFEAFFEECFF3FFEDCFF4FFEE2A97
:1096C000000EEF22F3CFE9FFF4CFEAFFFD0EDBCF70
:1096D000EFFFEF50016AF36E01C0F4FF10D0FB0EF4
:1096E000DB50FE0806E1FD0EDBCFE6FF65EC4CF03B
:1096F00005D0FD0EDBCFE6FF7CEC4CF0E552E552E9
:0A970000E5CFDAFFE7CFD9FF120032
:06970A003D504202F3CFC6
:1097100039F0F4CF3AF04302F3503A26000EF42029
:109720003B6E3D504402F3503B26000EF4203C6E4D
:109730003D504502F3503C263E504202F3503A263B
:10974000F4503B22000E3C223E504302F3503B2695
:10975000F4503C223E504402F3503C263F5042021B
:10976000F3503B26F4503C223F504302F3503C263A
:0A97700040504202F3503C26120064
:06977A0040C04AF03FC0B0
:1097800049F03F504402F4CF3EF0F3CF3DF040505B
:109790004502F4CF40F0F3CF3FF04402F3503E26B1
:1097A000F4503F22E86A402249504502F3503E26D9
:1097B000F4503F22E86A402245AEE3EF4BF04950B7
:1097C0003F5E4A50405A4AAE000C44503F5E4550FE
:0497D000405A000CEF
:0C97D4003C6A3B6A3A6A396A200EE76E74
:1097E000D8903D363E363F36403639363A363B36EF
:1097F0003C364250395C43503A5844503B584550EF
:109800003C5809E34250395E43503A5A44503B5A5F
:0C98100045503C5A3D2AE72EE4D71200D8
:04981C00D9CFE6FFBB
:10982000DACFE6FFE1CFD9FFE2CFDAFFACAC04D06C
:10983000AC900001FFB3AC80FD0EDB50AD6EE55285
:0A984000E5CFDAFFE7CFD9FF1200F1
:06984A00F36AF46AFF0E50
:10985000E124E96EFF0EE220EA6EED6607D02F0EDE
:0E986000EF6404D03A0EEF6001D0F32A12003C
:02986E00FF0EEB
:10987000E3504B6E480E01D04C0EE76EE72EFED73C
:0E988000E76AE72EFED74B2EF7D70000120046
:02988E00800E4A
:10989000F36E00EE00F00F0E01D81200EA6002D065
:0E98A000EE6AFCD7F350E9601200EE6AFCD7C6
:0298AE001EEEAC
:1098B00000F02EEE00F0F86A389CF4EC4AF07DECF3
:0A98C0004CF058EC30F0FBD712001A
:0698CA00FF0EE350ACBAF2
:1098D00004D0AF6AAB8EAC8A949CACA2FED7AD6EBE
:0698E000F36EF46A1200B1
:0A98E600303132333435363738396B
:0798F000616263646566001C
:0198F700FF71
:0298F80012005C
:0298FA0012005A
:0498FC002F6C6966FE
:10990000646174612E62696E20002F6870646973EF
:079910006B2E636667000087
:09991700800102E805000913407B
:109920000100010001F6008C119411941F01000048
:10993000000000000000000000E3400700000000FD
:109940003F005F0120016501200040003400370026
:0499500000000A0009
:0C99540080004C4142454C3100000002F4
:10996000800000000000000E00004D5946494C45A3
:1099700031323334000100000001000020001310D8
:0E9980001200000001000000000000000000C6
:020000040030CA
:0100010006F8
:0100020019E4
:010003001EDE
:010005008179
:010006008178
:00000001FF
